:10000000E264040000000000FFFFFF00FFFFFF00AC
:10001000FFFFFF00FFFFFF00FFFFFF00FFFFFF00EC
:10002000FFFFFF00FFFFFF00FFFFFF00580200007F
:10003000FFFFFF00FFFFFF0012020000FFFFFF00B5
:10004000FFFFFF00FFFFFF00FFFFFF0000010000B8
:10005000FFFFFF00AC020000FFFFFF00FFFFFF00FB
:10006000FFFFFF00FFFFFF00FFFFFF00BE010000DA
:100070006A010000FFFFFF00FFFFFF00FFFFFF001E
:10008000FFFFFF00FFFFFF00FFFFFF00FFFFFF007C
:10009000FFFFFF00FFFFFF00FFFFFF00FFFFFF006C
:1000A000FFFFFF00FFFFFF00FFFFFF00FFFFFF005C
:1000B000FFFFFF00FFFFFF00FFFFFF00FFFFFF004C
:1000C000FFFFFF00FFFFFF00FFFFFF00FFFFFF003C
:1000D000FFFFFF00FFFFFF00FFFFFF00FFFFFF002C
:1000E000FFFFFF00FFFFFF00FFFFFF00FFFFFF001C
:1000F000FFFFFF00FFFFFF00FFFFFF00FFFFFF000C
:10010000FFFFFF00FFFFFF00FFFFFF00FFFFFF00FB
:10011000FFFFFF00FFFFFF00FFFFFF00FFFFFF00EB
:10012000FFFFFF00FFFFFF00FFFFFF00FFFFFF00DB
:10013000FFFFFF00FFFFFF00FFFFFF00FFFFFF00CB
:10014000FFFFFF00FFFFFF00FFFFFF00FFFFFF00BB
:10015000FFFFFF00FFFFFF00FFFFFF00FFFFFF00AB
:10016000FFFFFF00FFFFFF00FFFFFF00FFFFFF009B
:10017000FFFFFF00FFFFFF00FFFFFF00FFFFFF008B
:10018000FFFFFF00FFFFFF00FFFFFF00FFFFFF007B
:10019000FFFFFF00FFFFFF00FFFFFF00FFFFFF006B
:1001A000FFFFFF00FFFFFF00FFFFFF00FFFFFF005B
:1001B000FFFFFF00FFFFFF00FFFFFF00FFFFFF004B
:1001C000FFFFFF00FFFFFF00FFFFFF00FFFFFF003B
:1001D000FFFFFF00FFFFFF00FFFFFF00FFFFFF002B
:1001E000FFFFFF00FFFFFF00FFFFFF00FFFFFF001B
:1001F000FFFFFF00FFFFFF00FFFFFF00FFFFFF000B
:100200003600F800801F7800200020000C00090054
:10021000B01F7800210480000020200000806000D2
:10022000C900DE000100E0002400320070108000F0
:1002300062006000C100DE006080500019003A00DA
:1002400001C0200020D0200090804000901080004D
:100250008048780010688000E10040001168880044
:10026000F00F20000080600010688800E10040006E
:10027000F00F20000081600001D02000110051002B
:1002800006003A00100020002068880000002000CE
:1002900000688800000020001068880058010400F1
:1002A00000000000D1FF2F00E02020001088600037
:1002B000F1DF2F004008200010886000A00120001E
:1002C0000C0009004F1078004F0078003600F9004C
:1002D000004006003600F800801F78002000200053
:1002E0000C000900B01F78008640AE00B201040087
:1002F000000000005E61AE00880104000000000004
:10030000E00A8000010020007A01040000000000E3
:10031000C1EF2000C8A2AE00980104000000000058
:100320008008780091009800B001040000000000EF
:100330000001780011005100306888008000EB0057
:1003400041688800516880000100E00004003A0024
:10035000616880000100E00001003200C00E8800EA
:100360008640A900A00120000C0009004F10780071
:100370004F0078003600F900004006003600F80013
:10038000801F7800200020000C000900B01F7800BA
:100390008620AE0006020400000000005A61AE0094
:1003A000DC01040000000000C00A80000100200001
:1003B000CE0104000000000081EF2000C882AE00E2
:1003C000EC01040000000000800878009100980013
:1003D0000402040000000000000178001100510038
:1003E000706888008000EB00816888005168800098
:1003F0000100E00004003A00616880000100E000B4
:1004000001003200B00E88008620A900A001200063
:100410000C0009004F1078004F0078003600F900FA
:10042000004006003600F800801F78002000200001
:100430000C000900B01F78008480AE004C0204005C
:10044000000000004661AE00300204000000000021
:10045000200A8000010020002202040000000000A9
:1004600001F02000D422AE00400204000000000091
:1004700080087800910098004A0204000000000003
:100480000001780011005100906888000000EB0026
:10049000A06888008480A900A00120000C00090049
:1004A0004F1078004F0078003600F9000040060039
:1004B0003600F800801F7800200020000C000900A2
:1004C000B01F78008420AE00A002040000000000ED
:1004D0004261AE007602040000000000000A8000C5
:1004E00001002000680204000000000041F020002C
:1004F000D402AE00860204000000000080087800EC
:10050000910098009E0204000000000000017800A5
:1005100011005100B06888008000EB00C1688800BD
:10052000516880000100E00004003A00616880002A
:100530000100E00001003200D00E88008420A900F4
:10054000A00120000C0009004F1078004F00780037
:100550003600F900004006003600F800801F7800E1
:10056000200020000C000900B01F7800210480004A
:100570000080200000806000CB00DE000100E00071
:100580002700320011158000000820000080600064
:10059000C700DE000100E0000800320010148000F7
:1005A000D068880020148000E06888000014800073
:1005B000F0688800EA020400000000009014800047
:1005C000D0688800A0148000E06888008014800053
:1005D000F0688800F168800000D220009080500010
:1005E000F16888006080500002003D00000020009B
:1005F000F0688800F16880004F89DE0020D220007A
:1006000010984000101049001100200060D2200016
:1006100010C84000F17F2F004008200010886000C3
:10062000A00120000C0009004F1078004F00780056
:100630003600F90000400600008823001100200069
:100640000000060001002800C02020001088700073
:1006500001402000E020200010887000000006000B
:10066000E0462000801F7800A0072000801F78004F
:10067000012E07004F00B100000006000000FA0044
:10068000711080000010200000806000C800DE00B3
:100690000100E00002003A004003040000000000F6
:1006A00068005700104078000080FB008010880030
:1006B0000080FA00000006000000000000000000BA
:1006C0009010800000000600701080006100600043
:1006D0000000060071108000001020000080600003
:1006E000C800DE000100E00003003A000000000046
:1006F0006A0304000000000000000600F1FF27006C
:10070000C020200010886000F1BF2F00E0202000F2
:1007100010886000000006000C00FA00E0332000A2
:1007200040698800C03520005069880040362000AC
:1007300060698800A036200070698800203220009F
:1007400080698800E0372000906988000000200060
:10075000601088000000280070108800B6FF0700B5
:10076000000F780011079800823E2000CF91DE0034
:10077000F02F07002007980031079800000F78003D
:100780001107980066002000CFB3DE006A02570010
:1007900034017800A40178000603E9000300350065
:1007A0000201D0008381D200FBFF3700420798008E
:1007B000530798000002EB002C1D07002E0290004A
:1007C000BE0290004E019000DE01900020079800CC
:1007D0003107980004007800850078000002EB00E3
:1007E0004E1D0700000F780011079800120020002E
:1007F000CF91DE004E009000DE00900000027800F5
:10080000810278000201E900030035008502D10071
:100810000482D300FBFF37002E019000BE01900040
:100820000400510005805900050036001200200028
:10083000CF91DE0060004700101841001090490081
:100840006001470032007800A2007800610050008B
:10085000E0805800000F780011079800A010880071
:10086000D2FF2F00E02020001008610075FF070074
:100870007BFF07007AFF07000080FA0000000600F7
:1008800040032000401588003030200030158800DB
:10089000C0042000001588002020200010158800CA
:1008A0007000200020158800F0FF2F00301688000F
:1008B00000002000A0168800F0FF2F00901688008E
:1008C00000002000C016880000002000F0168800FC
:1008D00000000600F1F32F00E020200010886000E7
:1008E000010120008009200090806800000720009E
:1008F000808060008009200010886800F1DF2F00F0
:10090000400820001088600001202000C00820005E
:1009100010887000000020003008880000012800C6
:1009200080088800606222007008880000002000B3
:100930005008880000022800900888000100280064
:10094000002A200010887000F17F2F00400820004E
:100950001088600001802000C0082000108870000E
:1009600001082000A0152000108870001100200050
:10097000A015200010806800E7006000A01520008E
:100980001088680001012000C009200090806800E4
:100990000007200080806000C009200010886800E7
:1009A000D1FF2F0060082000108860002100200087
:1009B000E00820001088700001082000E0152000E9
:1009C0001088700011002000E015200010806800E1
:1009D000E7006000E015200010886800011020008A
:1009E000C0092000908068000070200080806000B6
:1009F000C009200010886800B1FF2F0060082000A7
:100A00001088600041002000E0082000108870007D
:100A10000108200020142000108870001100200020
:100A20002014200010806800E700600020142000DF
:100A300010886800010120004009200090806800B3
:100A400000072000808060004009200010886800B6
:100A5000D1FF2F00400820001088600021002000F6
:100A6000C0082000108870000108200060142000D9
:100A700010887000110020006014200010806800B1
:100A8000E70060006014200010886800110020005A
:100A90006009200010806800E70060006009200005
:100AA00010886800F1FE2F004008200010886000C8
:100AB00001012000C008200010887000000006001E
:100AC0000200FA006800570010007800000F78005C
:100AD0009E0178001100200060004700108840004F
:100AE0003EB99700110020006A00570010884000AE
:100AF000924978001304E000020032006805040007
:100B0000000000004EB897000080FA0000000600C8
:100B10000000FA00F1FB2F00002220001088600086
:100B20000011800062006000C100DE000100E000F2
:100B30000200320090050400000000006800570029
:100B4000100078002011880000118000E100600092
:100B500002003A00A40504000000000020118000FB
:100B60000080FA00000006000000FA0001002800E2
:100B700000222000108870000080FA0000000600AB
:100B80000000FA00F1FF270000222000108860001A
:100B90000080FA00000006000000FA0080582000E3
:100BA000A0698800405B2000B0698800005C2000DC
:100BB000C069880068005700900078006A005700FC
:100BC000908070006C005700908070006E0057009D
:100BD0009080700070005700908070007200570085
:100BE000908070007400570010817000F60057006C
:100BF0002022200011087100F1FB2F0000222000AC
:100C00001088600001002800002220001088700079
:100C10000080FA00000006000C00FA0060004700A7
:100C2000810F2F000A00090031587800E0222000CF
:100C3000801F7800D0032000801F78008E2C0700D2
:100C40004F00B10060004700801F78007219070054
:100C50002F00B100E0462000801F7800A007200090
:100C6000801F7800842C07004F00B10068005700F7
:100C700010007800A01088000080FA000000060034
:100C80000200FA00F0FF2F00000F780014688000C7
:100C900003D02000130052000E00320003C02000D9
:100CA00000D0200090814100134078000080FB00BC
:100CB000000F780000688000E101400003688800B0
:100CC00002102000110009008281D8000100780084
:100CD000006888001E0078000080FA00000006000E
:100CE0001168800000D020001080500002003A00FF
:100CF0000000200001003700100020000000060066
:100D00000000FA006C0157009240780010002000AB
:100D1000124910000104E0001D0032004EB8970097
:100D20009040780060C05000070032003EB9970044
:100D30004EB897009040780012C0500002003A0070
:100D4000B806040000000000CEB897003EB8970037
:100D50001041780001007800904078008180FB000D
:100D60000281FB000200780000805000090037007B
:100D7000110020006800570010884000110020007A
:100D80006A0057001088400082060400000000003E
:100D9000000020000080FA00000006000400FA00B5
:100DA000680057001000780010079800000020002D
:100DB000000F7800620047009000780060805000CB
:100DC000110036001100200062004700108810005A
:100DD0001E017800110020006000470010884000CC
:100DE0006A0057001000410010417800C102200045
:100DF0000140510002003200E8060400000000003B
:100E0000DA060400000000001E0078000080FA00EE
:100E1000000006000600FA00CEB8970011407800E6
:100E20000080FB00000F780002022000E000470075
:100E300011001100060032006000470090007800A9
:100E400069805000020032003207040000000000F8
:100E50001100200068005700108840000C070400B3
:100E60000000000000002000100798000000200093
:100E700020079800D2022000E00047001100110076
:100E800008003A001100200064004700108840006C
:100E9000110020006800570010884000600704001F
:100EA00000000000B2022000E00047001100110025
:100EB00003003A001100200068005700108840002D
:100EC000CEB89700114078000080FB00000F78003A
:100ED00060004700901F7800BA1907002F00B1008A
:100EE0000000E0000D00320062024700940078002C
:100EF000A00020000089B900010320006000470025
:100F000010801000000A4100110020006800570006
:100F10001088400060070400000000002E009000D0
:100F20000000E0000400320062004700100078007A
:100F300060001000010037001E0090000080FA00E1
:100F4000000006002A00FA007000470031102F0050
:100F50001300090031587800000020003007980085
:100F60000000200001002000400798005107980071
:100F7000D0CC2C00C1DC23006007980071079800DA
:100F8000000020002017980000002000000F7800CB
:100F90006000470010017800730051001C003D0004
:100FA0006800570010017800600047001000410001
:100FB00010427800D2022000024052001400390092
:100FC00068005700100178006000470010004100E1
:100FD0001042780092032000024052000C003E00B4
:100FE00070004700E002470015024000680057000B
:100FF000100178000500780010004100104A7800C8
:1010000010002000950A4000C807040000000000FE
:10101000F0024700600247001481420000002000F7
:10102000004978000400780010007800100798004C
:101030000400780010007800200798000500780070
:1010400010427800D20220000240520002003A0012
:10105000100020003007980066004700100078005C
:10106000000F78006000470010027800620147001E
:101070001200520018003D00700147006000470058
:101080001000410010427800E202200002405200AD
:101090000C003A0060014700120078002007980019
:1010A000020078001002780066014700120052002A
:1010B00002003A00F0FF2F00200798006C0804009F
:1010C00000000000120020006000470010084100EE
:1010D0003208040000000000F4FF2F006401470004
:1010E000120012002A00320064004700100178004C
:1010F000600047006108510060004700100278005E
:101100006601470012005200210035006E00900079
:10111000FE0090000200200003122400FA2B0700BA
:1011200030179800411798006007980071079800E1
:101130007001470060004700100041001041780036
:101140000281FB000003200000005100CF80DE0080
:101150000081EB00912B07003E119000CE11900012
:10116000E92B07006802470034017800A4017800E9
:10117000BA2C070040079800510798001200200081
:1011800060004700100811007C0804000000000007
:101190000000200001F82300600798007107980004
:1011A00062004700100078006102500064014700AF
:1011B000120012003D003200F4FF2F0064014700CE
:1011C0001200120003003A00660047001000780089
:1011D00020079800000020002017980066004700B4
:1011E000100178006000510002003A001000200059
:1011F000201798006400470010017800660047003F
:101200001002410042022000020147006000470036
:101210001208420060004700100278006201470097
:101220001200520021003D000200200003122400A1
:101230006E009000FE009000472D070030179800C8
:1012400041179800600798007107980070014700E7
:101250006000470010004100104178000281FB004F
:101260000003200000005100CF80DE000081EB0071
:101270004A2B07003E119000CE119000A22B0700D0
:101280006802470034017800A4017800732C07003D
:1012900040079800510798001200200060004700A6
:1012A000100841000A090400000000006600470021
:1012B000100178006100510007003A004E009000D4
:1012C000DE0090000200200003F82B008E2B0700A8
:1012D00040079800510798004E009000DE009000F3
:1012E0000080FA00000006000800FA004EB99700DE
:1012F000124078000080FB00000F780004022000FC
:101300006001470012001200060032006000470032
:101310001001780069005100020032009C090400AD
:101320000000000012002000680057001008410073
:10133000760904000000000000002000CF80DE00DD
:10134000100798002107980000002000300798003F
:101350004EB8970010427800D2022000024052009E
:1013600008003A0012002000660047001008410003
:10137000120020006800570010084100D209040044
:10138000000000004EB8970010427800B202200022
:101390000240520003003A0012002000680057008B
:1013A000100841004EB99700124078000080FB0001
:1013B000000F780060004700901F78008118070038
:1013C0002F00B1000000E000120032001E0090006B
:1013D000AE009000A200200003002000D52C0700E2
:1013E000040320006001470012011200020278008D
:1013F000CFA2DE00620147000419400005914800B9
:10140000120020006800570010084100D2090400B3
:10141000000000003E0090000000E00006003200E6
:101420006200470030017800A001780060001100E0
:10143000E0801900020037001E009000AE0090000E
:101440000080FA00000006000000FA006A01570060
:10145000620041009040780020032000014878009D
:1014600012007800C00088009C05BA00B00080001F
:101470000080FA00000006000A00FA006A00570027
:1014800010007800100798004EB9970032007800DD
:10149000A200780020079800310798000000200083
:1014A000000F780060004700100278006C015700C0
:1014B0001200520015003D006400470040079800EC
:1014C000B01F7800A01F7800DFFF07004F00B100B9
:1014D0001E019000000978002200200062004700F1
:1014E0001008410022002000CF91DE004E00900045
:1014F00010184100109049001200200060004700C1
:1015000010084100520A0400000000006C0057005F
:10151000100078004100DD004EB99700CF80DE005A
:1015200012194000129148000080FA0000000600E5
:101530004E00FA006000470011132F00050009005B
:10154000315878006600470071132F00050009002C
:10155000315878006C004700D1132F0005000900B6
:10156000315878007200470031142F000400090040
:10157000315878007700470081142F0005000900DA
:10158000315878007D004700E1142F000600090063
:1015900031587800400220000000470051152F000C
:1015A000020009003158780000002000101F980048
:1015B00068005700901F7800F62307002F00B10045
:1015C0006200500040179800610150006800570009
:1015D0001000410010427800A20220000240520098
:1015E0000200320000002000D102370086022000F5
:1015F000060347001600780061005000680257009B
:101600001401400000002000004978000400780028
:1016100010017800060078001000410010417800A9
:101620000281FB00000320000001510052179800C6
:10163000690051000400340072002000A002200064
:101640000000470010081100A00220000000470021
:10165000100078004400DD00101F98008002200078
:10166000000047001000780061014000680057004A
:1016700010004100104178000281FB0000032000AF
:101680000001510052179800690051000400340015
:1016900072002000A0022000000047001008110086
:1016A000A002200000004700100178002003200065
:1016B000000047001008410000002000D0698800A9
:1016C00000002000501798000000200040179800EC
:1016D00068005700100178008002200000004700D9
:1016E0001000410010417800604051000E003200AF
:1016F00068005700100078008402200004024700B0
:1017000014004000104178000281FB00A00220007C
:10171000000047001008690010002000140A400073
:10172000680B0400000000002003200000004700B8
:1017300010027800A20220000201470012005200AD
:101740000400320010002000D06988000000200052
:101750007702370050002000801F78006800570093
:10176000901F780060004700801F780064FD07002C
:101770006F00B10060015000D2003A0068025700CB
:101780005427980014007800710040001041780040
:1017900070D220000248780004007800901F780082
:1017A00010002000801F78007CFD07004F00B10072
:1017B0004017980066014000680057001001410082
:1017C00000002000004978005E20900010017800A1
:1017D00080022000000047004027980010004100D0
:1017E00064004000801F78008AFD07002F00B100D0
:1017F000E0698800800220000000470010007800A7
:101800006401400068005700100141000000200002
:10181000004978005E209000100178004E20900072
:101820001000410062004000801F780079FD070031
:101830002F00B100F06988008002200000004700FE
:10184000100078006201400068005700100141005C
:1018500000002000004978005E2090001001780010
:101860004E20900010004100801F780069FD0700A5
:101870002F00B100006A880068005700901F7800B0
:1018800030002000801F780044FD07004F00B100A9
:1018900040179800680157001200400062004000A5
:1018A000801F7800A7FD07002F00B100201F9800BF
:1018B000311F9800800220000000470010007800CF
:1018C0006201400068005700100141000000200044
:1018D000004978005E209000100178004E209000B2
:1018E00010004100801F780096FD07002F00B10016
:1018F00020279800312798000200200003272400A9
:101900002E189000BE189000932B07002E219000F7
:10191000BE219000D12A0700106A8800216A880041
:1019200068005700901F780040002000801F78005A
:101930001AFD07004F00B100680157001200400077
:101940001041780060D42000024878005E209000AA
:10195000901F780050002000801F78000FFD0700C6
:101960004F00B10040179800680157001200400076
:1019700063004000801F780072FD07002F00B10057
:10198000201F9800311F98008002200000004700AF
:10199000100078006301400068005700100141000A
:1019A00000002000004978005E20900010017800BF
:1019B0004E20900010004100801F780061FD07005C
:1019C0002F00B10020279800312798000200200046
:1019D000032724002E189000BE1890005E2B0700ED
:1019E0002E219000BE2190009C2A0700406A8800AA
:1019F000516A880068005700901F7800600020003E
:101A0000801F7800E5FC07004F00B1006801570017
:101A1000120040001041780070D420000248780085
:101A20005E209000901F780070002000801F7800DA
:101A3000DAFC07004F00B1006801570012004000B7
:101A4000801F78003FFD07002F00B100606A88000A
:101A5000716A880068005700901F7800800020009D
:101A6000801F7800CDFC07004F00B10068015700CF
:101A700012004000801F780032FD07002F00B100E7
:101A8000806A8800916A880068005700901F78007B
:101A900090002000801F7800C0FC07004F00B100BC
:101AA0006801570012004000801F78000EFE0700FA
:101AB0002F00B100A06A8800B16A880010002000E1
:101AC0009B01370050002000801F780068005700FD
:101AD000901F780066004700801F780088FC070090
:101AE0006F00B1006001500028003A006800570004
:101AF000901F780070002000801F7800A7FC07006E
:101B00004F00B1006801570012004000801F7800AC
:101B1000C0FC07002F00B100C06A880068005700B1
:101B2000901F780080002000801F78009BFC070039
:101B30004F00B1006801570012004000801F78007C
:101B400000FD07002F00B100D06A8800E16A88001C
:101B500068005700901F780090002000801F7800D8
:101B60008EFC07004F00B1006801570012004000D2
:101B7000801F7800F3FC07002F00B100F06A880096
:101B8000016B880010002000690137005000200020
:101B9000801F780068005700901F78006C00470095
:101BA000801F780056FC07006F00B10060015000F4
:101BB000CF003A0010002000106B8800680057002A
:101BC000901F780030002000801F780073FC070011
:101BD0004F00B1006801570012004000801F7800DC
:101BE0008CFC07002F00B1005017980060015000D6
:101BF00004003D000000200050179800100E040063
:101C000000000000A0022000000047001001780042
:101C10006C00510002003400C000200050179800F2
:101C2000A002200000004700100078004017980034
:101C3000A002200000004700100178006C00510055
:101C400016003D00A40220000402470014007800A2
:101C50004201DD0040D620000201400000002000CB
:101C60000009780004007800100078004201DD00CF
:101C700040D6200002004000620140000000200029
:101C80000009780012002000A00220000000470098
:101C900010084100180E0400000000006800570002
:101CA000901F780020002000801F78003BFC070078
:101CB0004F00B1006801570012004000801F7800FB
:101CC00054FC07002F00B10061015000621798001A
:101CD0006300510084003D00C00220000000470066
:101CE000100078004201DD00800220000000470063
:101CF00010011100421798006400510002003400E6
:101D00004000200040179800000020005017980065
:101D1000A00220000000470010027800820220008C
:101D200002014700120052006F003D00680057009A
:101D3000901F7800A00220000000470010007800EB
:101D40004200DD0064004000801F780013FC0700A3
:101D50004F00B100101F98006801570012004000AA
:101D6000104178006040510059003200680057006F
:101D700010017800200320000000470010004100FF
:101D800010427800C202200002405200500032008F
:101D9000C002200000004700602798001000780073
:101DA0004201DD00A00220000000470050279800FB
:101DB000100041004201DD0040D62000020040003A
:101DC00040279800680057002027980010017800ED
:101DD000200320000000470010004100801F780011
:101DE0000CFC07002F00B1004E2190000009780084
:101DF0002E209000901F78005E2090001000780048
:101E00004200DD006400400063004000801F780055
:101E1000E2FB07004F00B100101F9800C202200033
:101E200002014700120178004212DD00A2022000E8
:101E300002014700120142004212DD0042D620009A
:101E40000401410062014100222798006801570007
:101E500012004000801F7800EEFB07002F00B10049
:101E60004101DD002E209000020878006E209000D5
:101E7000100078004201DD005E209000100041005B
:101E80004201DD0040D62000020040006202400016
:101E900032062000140011000D003600C0022000A0
:101EA00000004700100078004201DD00A002200081
:101EB00000004700100041004201DD0040D6200034
:101EC0000200400062014000300620000009780056
:101ED00012002000A002200000004700100841006E
:101EE000880E040000000000100020009000370061
:101EF00050002000801F780068005700901F780075
:101F000072004700801F78007DFB07006F00B10062
:101F10006001500006003A0077004700801F7800FB
:101F20009E1407002F00B100100020008000370031
:101F300050002000801F780068005700901F780034
:101F40007D004700801F78006DFB07006F00B10027
:101F50006001500073003A0080C52F00F107200097
:101F6000002798001127980010002000801F78009B
:101F7000A002200000004700801F7800000420001D
:101F800000004700801F78003BFD07006F00B10094
:101F900020002000801F7800E002200000004700A1
:101FA000801F78000004200000004700801F780098
:101FB00031FD07006F00B100E00220000000470083
:101FC000B01F7800A01F780070112F00801F7800CC
:101FD00040D92000801F78005C2107008F00B100ED
:101FE00040D92000801F78006C1407002F00B1003A
:101FF0005E12900012002000A002200000004700A6
:1020000010081100600052003F003400000420005E
:102010000000470030027800A002780042FF2F0045
:10202000F30720000200520003805A0036003E00F1
:1020300020002000801F780080032000000047005F
:10204000801F78000004200000004700801F7800F7
:1020500009FD07006F00B10020002000801F7800FC
:10206000C003200000004700801F7800000420000B
:1020700000004700801F7800FFFC07006F00B100E0
:1020800010002000801F7800800220000000470020
:10209000801F78000004200000004700801F7800A7
:1020A000F5FC07006F00B10080022000000047002F
:1020B000901F7800C003200000004700B01F780088
:1020C000A01F78008003200000004700B01F7800A8
:1020D000A01F780010122F00801F780040D9200028
:1020E000801F780019210700EF00B10040D92000BF
:1020F000801F7800291407002F00B1000060FE0047
:10210000F80F04000000000040022000000047001B
:10211000801F7800211407002F00B100100020005C
:102120000300370020002000D06988000000200054
:102130000080FA00000006000000FA00806E8000B7
:102140000000E0001100320068005700901F780086
:10215000102107002F00B1008102200000805000F4
:10216000C180DE00906E800068004000801F780013
:10217000811F78005F0907004F00B1006800570019
:10218000901F7800162107002F00B1000080FA0090
:10219000000006001000FA0060004700A1162F00A2
:1021A0000C00090031587800D06A8000E16A800094
:1021B0000200200003002000602807000000E0006B
:1021C00002003C0000002000010037001000200049
:1021D0000000E00056003200D26A8000E36A80000E
:1021E000A06E8000B16E8000542807000000E0005F
:1021F00002003D0000002000010037001000200018
:102200000000E0004A003200D06A8000E16A8000ED
:10221000A06E8800B16E8800C26E80006000510020
:1022200033003C00806E80000000E00001003200BE
:102230005C110700406A8000516A8000D06E8800FF
:10224000E16E8800106A8000216A8000F06E8800CC
:10225000016F8800F06A8000016B8000106F8800B9
:10226000216F880060D420001042780032052000E1
:102270000240520005003A0002002000030028003E
:10228000E0DD2000101869001090690070D4200073
:1022900010427800720520000240520005003A000A
:1022A0000200200003002800A0DD200010186900B3
:1022B00010906900006A8000F06F8800F06980006B
:1022C00000708800E0698000107088001000200015
:1022D0002070880000002000801F7800171407007D
:1022E0002F00B100EC200700941104000000000052
:1022F000C06E800061005000C06E8800801F7800B2
:1023000080152F00801F780040D92000801F7800A2
:102310008E2007006F00B10040D92000801F780098
:1023200085FF07002F00B100E61104000000000047
:10233000C46E800062E02000120052001F003200D4
:1023400000002000700798006E0047001001780020
:10235000760051000A003D0042D920006E0047007F
:102360001001410000022000004978001200200006
:102370006E00470010084100A41104000000000096
:1023800042D920006E0047001001410000002000EB
:102390000049780040D92000801F780066FF0700C0
:1023A0002F00B10030708000C06E880060004700D0
:1023B000801F780060FF07002F00B1004070800090
:1023C00051708000A06E8800B16E88000080FA0015
:1023D000000006000800FA006A005700B01F7800ED
:1023E000A01F7800A70307004F00B100000178008C
:1023F000810178000000200001F823001228070066
:102400000000E0000200350000002000010037005D
:10241000100020000000E000030032000000200057
:10242000010020006D0037003EB89700CEB897003D
:102430003EB99700CEB997003327070020079800D0
:10244000310798000000200001F82300821F780067
:10245000831F78002E019000BE019000BC2707006A
:102460004F01BE00801F7800811F78005D000700CB
:102470004F00B100000F7800110798006A00570064
:10248000B01F7800A01F78007E0307004F00B10046
:102490000001780081017800F0282C0051F323001E
:1024A000A62707000000E00002003C00000020001A
:1024B00001003700100020000000E0000A00320098
:1024C0001E0178009E0190003EB89700CEB897009C
:1024D000A1280700801F7800811F7800A70307004C
:1024E0004F00B1003D0037006A015700320078000C
:1024F000A20078000200200003002000D22707007D
:102500000000E0000200350000002000010037005C
:10251000100020000000E0001D00320060004700B5
:1025200030017800A00178000000200001002800A0
:1025300000006900818069003EB99700CEB997001C
:1025400085280700801F7800811F78008B03070013
:102550004F00B1002007980031079800B0FD20001F
:1025600091FC2300821F7800831F78002E019000C9
:10257000BE019000762707004F01BE000200200038
:102580000300280002006800838068001300370001
:102590003EB99700CEB997001E0078009E009000CB
:1025A0006D280700801F7800811F780073030700E3
:1025B0004F00B1002007980031079800B0FD2000BF
:1025C00091FC2300821F7800831F78002E01900069
:1025D000BE0190005E2707004F01BE000080FA0098
:1025E000000006000E00FA006A0157003200780071
:1025F000A2007800020020000300200092270700BC
:102600000000E0000200340000002000010037005C
:10261000100020000000E000030032000000200055
:10262000010020006F0037006A0157003200780077
:10263000A2007800000F78001107980002007800CF
:1026400030017800A00178000000200001F823008C
:102650003A2707000000E00002003C0000002000D4
:1026600001003700100020000000E00007003200E9
:102670001E0178009E0190000000200001F8230058
:1026800035280700000F7800110798006A004700FE
:10269000801F780060004700B01F7800A01F7800FE
:1026A000520007006F00B100000F7800110798007A
:1026B0006A014700120178004191DE00821F780014
:1026C000801F7800811F78009C0007006F00B10018
:1026D000000F7800110798006A0057003001780059
:1026E000A00178000000200001F823001327070054
:1026F0000000E00002003C00000020000100370064
:10270000100020000000E000070032001E017800E9
:102710009E0190000000200001F823000E28070011
:10272000000F780011079800400120004007980032
:102730001E0178009E0190003EB89700CEB8970029
:1027400005280700600247006407980034017800FC
:10275000A4017800412707000200200003002400A4
:10276000FD27070020079800310798000002780035
:10277000810278006E00900000017800320078003D
:10278000A200780004017800850178002E27070058
:102790000000E000020032000000200001003700CD
:1027A000100020000000E00002003200EE130400E0
:1027B000000000006401470032007800A2007800A9
:1027C000000F78001107980068004700100078009B
:1027D0006101500042079800D5FF3A001E007800C2
:1027E0009E0090000080FA00000006000400FA003D
:1027F000600247006A01570032007800A2007800AA
:10280000001A78000112780062004200100178007E
:1028100000F8270000006100C701DE00E207200089
:102820002EB8970002885100E201420000F0230018
:102830001301680000F82700000061009309680098
:1028400034007800A40078000080FA000000060040
:102850000600FA006A01570032007800A2007800F2
:102860000200200003002000F72607000000E0001F
:10287000020034000000200001003700100020009A
:102880000000E000030032000000200001002000F2
:102890002800370060004700801F78006A0057005A
:1028A000B01F7800A01F7800D0FF07006F00B100B4
:1028B000020020000300240013260700020020006D
:1028C00003F82300A226070030BF9F0041BF9F00EE
:1028D000140020006001470012091200820020004D
:1028E000821F780082172F00821F7800801F7800D7
:1028F000811F78007D0207008F00B100100798004B
:102900002107980030BF9F0041BF9F001E00780044
:10291000CF80DE000081EB00A02507008221270088
:1029200013F32300F82507001E019000AE0190006C
:10293000CA2607000080FA00000006000400FA0022
:10294000E00147006A01570032007800A2007800D9
:1029500080197800811178006280410010017800B0
:1029600000F82700000061004701DE006C005700FE
:102970001001410022BF9F006000510003003D0094
:10298000000020000100200023003700F30F20008A
:102990006C01570012801100130034006A015700C7
:1029A00032007800A200780002002000030020001E
:1029B000A52607000000E00002003500000020000E
:1029C00001003700100020000000E000030032008A
:1029D000F0FF2F00F1F72F000F003700F0FF2F005E
:1029E000F1F727000C00370060004700E2014000CB
:1029F0006C005700100078004700DD0013016800EC
:102A000000F827000000610093096800600147009A
:102A100032007800A20078000080FA000000060072
:102A20000800FA006A01570032007800A20078001E
:102A30000200200003002000832607000000E000C1
:102A400002003200000020000100370010002000CA
:102A50000000E000030032000000200001F8230025
:102A60007B0037006A00570030017800A001780031
:102A7000E04F2D00212B2400732607000000E0000A
:102A80000200350000002000010037001000200087
:102A90000000E00003003200F0FF2F00F1F72700F4
:102AA0006B0037006A00570030017800A001780001
:102AB00000C52A00E12A2C00202607000000E000C3
:102AC00002003C0000002000010037001000200040
:102AD0000000E000030032000000200001002000A0
:102AE0005B0037006A01570032007800A2007800CE
:102AF0000200200003002000532607000000E00031
:102B00000200350000002000010037001000200006
:102B1000000F78000000E0000500320002002000F5
:102B2000030028006A00570010186900109069001F
:102B30003EB89700CEB89700B2A32A0083FB2300CB
:102B40007125070030BF9F0041BF9F00801F7800A4
:102B5000811F7800B30007004F00B100D3240700A5
:102B600030079800CF80DE000081EB000B250700C6
:102B700010079800210798006A015700320078007A
:102B8000A2007800821F7800831F78001E01900049
:102B9000AE019000EE2507004F01BE0030BF9F0040
:102BA00041BF9F003E019000821F780092002000EC
:102BB000821F7800C2192F00821F7800801F7800C2
:102BC000811F7800C90107008F00B100801F7800C5
:102BD000811F780059FF07006F00B10030BF9F00D0
:102BE00041BF9F001E0078000000E0001600320088
:102BF0006A00570030017800A0017800F0FF2F0034
:102C0000F1F72700102607000000E0000200320064
:102C10000000200001003700100020000000E0004C
:102C200003003200000020000100200008003700EF
:102C30003EB99700CEB997000000200001F82300AC
:102C4000C5260700020037003EB89700CEB89700AF
:102C50000080FA00000006000600FA0000002000D4
:102C6000000F78006A01570032007800A200780057
:102C70000200200003002000F32507000000E00010
:102C80000200320000002000010037001000200088
:102C90000000E000030032000000200001002000DE
:102CA0005E0037006E01570032007800A200780005
:102CB0000200200003002000E32507000000E000E0
:102CC0000200320000002000010037001000200048
:102CD0000000E000030032000000200001F82300A3
:102CE0004E0037006A01570032007800A2007800D9
:102CF0000200200003002000D32507000000E000B0
:102D00000200350000002000010037001000200004
:102D10000000E000220032001EB89700AEB8970015
:102D20009C13070010079800210798000001EB0092
:102D30009A24070000027800810278006E01570093
:102D400032007800A2007800040178008501780044
:102D5000BD2507000000E00002003A00000020004E
:102D600001003700100020000000E00003003200E6
:102D7000000020000100200028003700620047000A
:102D80001001780060004700610861000200200027
:102D9000030028006A0057001018690010906900AD
:102DA0006A005700B01F7800A01F7800A8FE070037
:102DB0004F00B10030BF9F0041BF9F001EB9970078
:102DC000AEB99700D024070030BF9F0041BF9F00DD
:102DD000801F7800811F780011FF07004F00B100AD
:102DE00030BF9F0041BF9F001E0078000000E00040
:102DF000080032006A00570030017800A001780016
:102E000000002000010028000000690081806900A6
:102E1000020037003EB89700CEB897000080FA0055
:102E2000000006000600FA006A0357007001200047
:102E3000CF80DE0036027800A60278000000E900AC
:102E4000030035008502D1000482D300FBFF370068
:102E5000F00F20000002620024079800F007200015
:102E600000025200240798006000520013003D0049
:102E70006A02570034007800A400780002002000A5
:102E800003002000702507000000E000020035006C
:102E90000000200001003700100020000000E000CA
:102EA000030032000000200001F82B002B00370047
:102EB00000002000010020002800370064004700C7
:102EC0001002780078005200030036003EB89700E8
:102ED000CEB89700210037003EB89700CEB89700D3
:102EE000F22307000081EB002C240700000F78007C
:102EF0001107980000037800810378006A025700E8
:102F000034007800A400780006017800870178007A
:102F10004D2507000000E000020035000000200001
:102F200001003700100020000000E000090032001E
:102F30006000470030027800A00278000200200004
:102F400003F82300040078008500780000250700BE
:102F5000020037001E0078009E0090000080FA00FA
:102F6000000006000A00FA00000020002007980078
:102F70006A02570034007800A400780002002000A4
:102F800003002000302507000000E00002003500AB
:102F90000000200001003700100020000000E000C9
:102FA0000700320004002000050028006A005700D6
:102FB00010186A0010906A00100020002007980086
:102FC0003EB89700CEB8970032982F0023E2230036
:102FD0004D24070030BF9F0041BF9F00801F780035
:102FE000811F78008FFF07004F00B1003007980065
:102FF000410798006A02570034007800A400780066
:10300000821F7800831F78003E019000CE0190005F
:10301000CF2407004F01BE00020020000308240057
:103020003924070030BF9F0041BF9F000002780095
:1030300081027800000020000100240004017800D3
:1030400085017800002507000000E000020035003F
:103050000000200001003700100020000000E00008
:10306000110032006A00570030027800A002780098
:10307000020020000300240004007800850078008E
:10308000B324070030BF9F0041BF9F002E00900077
:103090000000E000020032000000200001003700C4
:1030A00010002000200798006A00570030027800C6
:1030B000A00278000000200001F82300040178003D
:1030C00085017800E02407000000E00002003500E0
:1030D0000000200001003700100020000000E00088
:1030E0000A00320006002000070024006A02570090
:1030F00034017800A4017800060078008700780089
:103100009324070030BF9F0041BF9F003EB8970047
:10311000CEB897003EB99700CEB99700FA230700C2
:10312000000F78001107980044002000841F7800E9
:10313000441C2F00841F7800801F7800811F7800B6
:103140006A0007008F00B1003EB99700CEB9970022
:10315000ED23070030BF9F0041BF9F0030002000DB
:10316000801F7800801D2F00801F780060004700BE
:10317000B01F7800A01F78005C0007008F00B1002E
:1031800000017800810178003EB89700CEB8970022
:103190007125070030BF9F0041BF9F002E009000A7
:1031A0000000E000080032006A005700300278009A
:1031B000A0027800000020000100280000006A0042
:1031C00081806A00020037003EB89700CEB89700B1
:1031D0000080FA00000006000000FA006A005700B4
:1031E00030027800A0027800B0FD20009104240095
:1031F0000401780085017800932407000000E000B6
:1032000002003500000020000100370010002000FF
:103210000000E0000D0032006A0057003002780024
:10322000A002780042BE2C0063092400040078004C
:103230008500780046240700801F7800811F7800F1
:1032400048FF07004F00B1000C0037006A0057002C
:1032500030027800A0027800B0FD200091FC23002D
:1032600004017800850178007C240700801F780025
:10327000811F78003BFF07004F00B1000080FA007B
:10328000000006000000FA006A01570032007800D2
:10329000A200780002002000030020006A2407003A
:1032A0000000E000020035000000200001003700AF
:1032B000100020000000E000080032006A00570003
:1032C00030017800A00178000000200001002800F3
:1032D0000000690081806900020037003EB8970055
:1032E000CEB897000080FA00000006000400FA0043
:1032F0006E005700100078004201DD006C0057009E
:103300001001410032007800A2007800000F780020
:10331000110798001EB897000000E000130032006B
:103320003EB89700CEB897001E0178009E0190002D
:10333000752307006E0157001201780061015100EA
:1033400012BF9F004212DD006C01570012024200C2
:1033500034017800A401780040240700000F7800B1
:10336000110798008A190400000000001E00780070
:103370009E0090000080FA00000006000A00FA009B
:103380006A005700B01F7800A01F7800BDFF07003B
:103390004F00B1001007980021079800020020009C
:1033A00003002000282407000000E0000200320093
:1033B0000000200001003700100020000000E000A5
:1033C0000300320000002000010020006B003700E5
:1033D0006200470030027800A00278000000200060
:1033E00001F8230004017800850178001624070005
:1033F0000000E0000200350000002000010037005E
:1034000010002000000F78000000E00007003200EC
:103410001E019000AE0190000000200001F8230082
:10342000CD24070010079800210798001E00900087
:10343000AE0090001E019000AE0190003223070004
:10344000300798004107980054002000841F78003E
:10345000841E2F00841F7800801F7800811F780051
:10346000A2FF07008F00B1001E019000AE01900086
:10347000252307001007980021079800400020002E
:10348000801F780000202F00801F78006600470012
:10349000B01F7800A01F780094FF07008F00B100D4
:1034A00000017800810178001E009000AE009000BD
:1034B000A924070010079800210798001E00780033
:1034C0000000E0000A003200B6FD200097FC230057
:1034D0006202470034017800A401780006007800F9
:1034E000870078009A2307001007980021079800AA
:1034F0006A02570034007800A4007800020020001F
:1035000003002000D02307000000E0000200350087
:103510000000200001003700100020000000E00043
:103520000B0032006200470030027800A0027800F1
:10353000000020000100280000006A0081806A006D
:103540000003780081037800B21A04000000000034
:103550006202470034007800A4007800000378007D
:103560008103780006007800870078001007980033
:10357000210798001E009000AE0090000080FA0025
:10358000000006000000FA006E01570032007800CB
:10359000A20078000200200003002000672307003B
:1035A0000000E00002003C000000200001003700A5
:1035B000100020000000E0000A0032001EB9970051
:1035C000AEB997003EB89700CEB8970062240700C6
:1035D000801F7800811F780068FF07004F00B1004E
:1035E0007D0037006A01570032007800A2007800A1
:1035F0000200200003002000502307000000E0002C
:1036000002003D00000020000100370010002000F3
:103610000000E0001A0032006E015700320078000E
:10362000A20078000200200003002000862307008B
:103630000000E0000200350000002000010037001B
:10364000100020000000E0000D0032001EB99700BD
:10365000AEB997003EB89700CEB897003E24070059
:10366000801F7800811F780044FF07004F00B100E1
:10367000B2FD200093042400782307005600370091
:103680006A01570032007800A20078000200200092
:10369000030020006C2307000000E000020035005A
:1036A0000000200001003700100020000000E000B2
:1036B0002A0032006E01570032007800A200780024
:1036C00002002000030020005F2307000000E0004C
:1036D000020035000000200001003700100020002B
:1036E0000000E0000D0032001EB99700AEB997004F
:1036F0003EB89700CEB8970017240700801F7800C7
:10370000811F78001DFF07004F00B100B2FD2000AF
:1037100093042C00512307002F0037006E0157003F
:1037200032007800A2007800020020000300200090
:10373000452307000000E0000200320000002000E6
:1037400001003700100020000000E00003003200FC
:10375000B0FD200091FC2B001F0037006E015700C8
:1037600032007800A2007800020020000300200050
:10377000352307000000E0000200320000002000B6
:1037800001003700100020000000E00010003200AF
:103790006A01570032007800A20078000200200081
:1037A00003002000E52207000000E00002003C00CA
:1037B0000000200001003700100020000000E000A1
:1037C00003003200B0FD200091FC2300020037000E
:1037D00000002000010020000080FA000000060028
:1037E0001800FA00406A8000516A8000B2FD200093
:1037F00093042400442207000200200043332400E5
:10380000D5230700000F780011079800106A800088
:10381000216A8000B2FD2000930424003A220700B0
:103820000200200043332400CB2307004007980008
:103830005107980070D420001043780074052000D0
:103840000440530005003A00040020000500280051
:103850006000470010186A0010906A0060D42000D1
:1038600010437800340520000440530005003A005E
:1038700004002000050028006800470010186A00B6
:1038800010906A0024012000680057001022B80040
:10389000A0DD200004024000040F980034007800EE
:1038A000A4007800B2FD2000930424001622070033
:1038B0000200200043332400A723070020079800BC
:1038C000310798000E089000640240003400780030
:1038D000A4007800B2FD2000930424000A2207000F
:1038E00002002000433324009B2307006007980058
:1038F000710798000400200005002400841F780050
:10390000851F78006803470036027800A602780019
:1039100004017800850178008D2207000200200054
:10392000030024008C230700801F7800811F78008B
:103930008CFD07004F00B100801F7800811F7800C8
:10394000C5FC07008F00B100200F9800310F9800D0
:1039500068004700B01F7800A01F78001EFE070017
:103960004F00B100000F9800110F98006C00470045
:10397000B01F7800A01F780017FE07004F00B100AD
:103980000E0A90009E0A90000401780085017800DC
:10399000DD210700000F9800110F980000002000A3
:1039A00001002400801F7800811F78006400470018
:1039B00030037800A00378006002470034017800EB
:1039C000A4017800060078008700780060220700D4
:1039D00002002000030024005F230700801F7800FE
:1039E000811F78005FFD07004F00B100801F780045
:1039F000811F780098FC07008F00B1000E0A90002C
:103A00009E0A90000401780085017800BE2107001D
:103A10002E0A9000BE0A900004017800850178000B
:103A20008E220700801F7800811F7800EDFA0700C2
:103A30004F00B100801F7800811F780065FA0700F1
:103A40004F00B1000200200003002400AE21070057
:103A50000200200043332400AB210700B2FD200008
:103A6000930424003C23070002002600A3762400D0
:103A7000A521070062E52000D3FE2300A221070054
:103A80006070880071708800040020000500240028
:103A9000841F7800851F7800801F7800811F7800C0
:103AA0006DFC07008F00B100000F9800110F980007
:103AB0000000200001002400801F7800811F780092
:103AC000140EF800160EF80063FC07008F00B1001A
:103AD0000E0A90009E0A900004017800850178008B
:103AE0005E220700801F7800811F7800BDFA070062
:103AF0004F00B10080708800917088006800470016
:103B0000B01F7800A01F7800B3FD07004F00B10080
:103B1000000F9800110F98006C004700B01F78004C
:103B2000A01F78000FFD07004F00B1000E0A9000A3
:103B30009E0A900004017800850178007221070038
:103B4000200F9800310F980068004700B01F7800E0
:103B5000A01F780003FD07004F00B100000F980080
:103B6000110F98006C004700B01F7800A01F78006C
:103B700099FD07004F00B1000E0A90009E0A9000C8
:103B800004017800850178005F210700000F98008C
:103B9000110F98006400470030037800A0037800FC
:103BA0006002470034017800A40178000600780024
:103BB00087007800E6210700801F7800811F7800C9
:103BC00085FD07004F00B1000E0A90009E0A90008C
:103BD00004017800850178004B210700000F980050
:103BE000110F98002E089000BE089000821F7800E8
:103BF000831F78000E0990009E099000D4210700D1
:103C00004F01BE00801F7800811F780064004700CC
:103C100030037800A0037800600247003401780088
:103C2000A40178000600780087007800C82107000A
:103C3000801F7800811F7800CAFC07004F00B10088
:103C4000000F9800110F98006C004700B01F78001B
:103C5000A01F780060FD07004F00B1000E0A900021
:103C60009E0A900004017800850178002621070053
:103C7000801F7800811F780042FE07008F00B1008E
:103C800002002000433324001F210700B2FD200062
:103C900093042400B0220700C0708800D17088000F
:103CA0000200200003002000E72107000000E000E0
:103CB0000200350000002000010037001000200045
:103CC0000000E0000900320004002000453B240011
:103CD000C0708000D17080000401780085017800F8
:103CE000DE210700C0708800D1708800000020002D
:103CF000F070880000002000E0708800E469800017
:103D000020E0200010025200047188006000520080
:103D100006003D00C403200000E22000100842001D
:103D200014002000E0E1200010081200F469800077
:103D300000E0200010025200E0E1200010024200EA
:103D4000F47088006000520006003D00C4032000AB
:103D5000E0E120001008420014002000C0E1200033
:103D600010081200046A8000E0DF200010025200F8
:103D7000C0E1200010024200E470880060005200A0
:103D800003003D0084012000C0E120001008420033
:103D9000C46A80006300520036003400646A800008
:103DA000756A800010718000217180000401780024
:103DB00085017800A42107000000E0000200350022
:103DC0000000200001003700100020000000E0008B
:103DD00004003200606A8000716A800010718800FF
:103DE000217188008470800095708000307180009F
:103DF000417180000401780085017800922107005C
:103E00000000E00002003500000020000100370043
:103E1000100020000000E0000400320080708000EC
:103E2000917080003071880041718800A47080001A
:103E3000B5708000507180006171800004017800CD
:103E400085017800802107000000E00002003500B5
:103E50000000200001003700100020000000E000FA
:103E600004003200A0708000B170800050718800A2
:103E7000617188000080FA00000006002A00FA0044
:103E80006000470041212F000400090031587800EC
:103E90006500470091212F000E000900315878007D
:103EA00020032000200F98006800570010027800BF
:103EB0006000520015003A00707180000000E000C0
:103EC00010003200000020009071880000002000E7
:103ED0008071880000002000707188007400470025
:103EE000901F7800700B2000801F7800DF01070012
:103EF0004F00B10060004700801F7800B81907002C
:103F00002F00B100982204000000000074718000AE
:103F1000600052000C003A00100020007071880010
:103F200074004700901F7800700B2000801F7800FD
:103F3000CE0107004F00B10065004700801F7800E8
:103F4000A71907002F00B1006A005700100278007F
:103F50006100520050013500A4718000B5718000ED
:103F6000A2708000B37080000400780085007800A3
:103F7000F7200700300F9800410F980000027800EA
:103F800081027800C0718000D17180000401780046
:103F9000850178002C2107000000E00002003500B8
:103FA0000000200001003700100020000000E000A9
:103FB00006003200C0718000D1718000300F98007F
:103FC000410F98001E20040000000000C471800012
:103FD000D5718000000020000100280000036A0065
:103FE00081836A007600470030027800A0027800E2
:103FF00006007800870078000401780085017800C9
:10400000CE2007000000E00002003C00000020007D
:1040100001003700100020000000E000070032001F
:10402000C6718000D77180000400200005002800C0
:104030007600470004186B0005906B003E08900066
:10404000CE089000E2718000F37180002E200700FE
:10405000700F980001179800000278008102780024
:1040600000728000117280000401780085017800E0
:10407000F52007000000E0000200350000002000ED
:1040800001003700100020000000E00006003200B0
:104090000072800011728000700F98000117980064
:1040A0008C20040000000000047280001572800063
:1040B000000020000100280000036A0081836A00DC
:1040C0007E00470030027800A002780006007800E9
:1040D00087007800040178008501780097200700A8
:1040E0000000E00002003C0000002000010037005A
:1040F000100020000000E00007003200067280007F
:104100001772800004002000050028007E00470090
:1041100004186B0005906B00646A8000756A80006B
:1041200020728000317280000401780085017800DF
:10413000822007000000E00002003C000000200098
:1041400001003700100020000000E0000A003200EB
:104150002272800033728000606A8000716A800081
:104160007D2107007E0990008E119000E61F070058
:10417000700F980001179800C4708000D5708000FF
:10418000826A8000936A80000400780085007800CD
:104190006F200700500F9800610F98000002780010
:1041A00081027800000020004133240004017800DF
:1041B00085017800A42007000000E000020035001F
:1041C0000000200001003700100020000000E00087
:1041D0000C00320006002000473B24007A02470012
:1041E00034017800A4017800060078008700780088
:1041F00057200700500F9800610F980034210400E9
:10420000000000007A00470030027800A002780029
:104210000000200041332C00040178008501780063
:10422000462007000000E00002003C0000002000E3
:1042300001003700100020000000E0000A003200FA
:104240007A00470030027800A002780000002000C9
:10425000413B240004017800850178007F2007009D
:10426000500F9800610F98007A00470030027800E4
:10427000A0027800000020004123240004017800FF
:1042800085017800702007000000E0000200350082
:104290000000200001003700100020000000E000B6
:1042A000060032000000200041232400500F980037
:1042B000610F980084210400000000007A0047008C
:1042C00030027800A00278000000200041232C007A
:1042D0000401780085017800182007000000E00044
:1042E00002003C0000002000010037001000200008
:1042F0000000E000040032000000200041232C00F8
:10430000500F9800610F98000200200043332400F2
:104310005E089000EE0890000F21070042728000B6
:1043200053728000781F070010179800211798001B
:1043300000027800810278000000200001172400AC
:1043400004017800850178003F2007000000E000AC
:10435000020035000000200001003700100020009E
:104360000000E000060032000000200001172400D9
:104370001017980021179800E821040000000000A1
:10438000200220000000470030027800A0027800E0
:104390000000200001172C0004017800850178003E
:1043A000E61F07000000E00002003C0000002000C3
:1043B00001003700100020000000E000040032007F
:1043C0000000200001172C001017980021179800FA
:1043D0007E00470030027800A002780072728000F0
:1043E000837280000400780085007800D81F0700E1
:1043F000AE1E070060728800C61220000602500040
:1044000004003400C01220006072880016220400EC
:10441000000000006672800044ED2F00040053008D
:1044200002003D0040ED2F00607288002002200055
:104430000000470030027800A0027800A2728000DD
:10444000B37280000400780085007800C01F070068
:1044500002002000031024002B1F0700931E0700FA
:1044600090728800C612200006025000040034003A
:10447000C0122000907288004C220400000000004E
:104480009672800044ED2F000400530002003D00AE
:1044900040ED2F00907288006472800000E32000DD
:1044A000301798001002520032002000110009005D
:1044B0000202D8003E1290001400400040179800FD
:1044C000807188009472800020E3200030179800EB
:1044D0001002520032002000110009000202D80030
:1044E0003E1290001403400096718800A4E520005D
:1044F0004E1090001484B900C8728800E0E52000D6
:1045000010B3B900E672880006738800E4D020007A
:10451000601D20001408140064D02000801D2000BD
:104520001408430064D12000A01D200014081300CB
:104530000080FA00000006000E00FA0080C52F007F
:10454000F10720004007980051079800406A80005A
:10455000516A8000000F780011079800106A8000EF
:10456000216A8000200798003107980060D420005D
:1045700010427800320520000240520005003A0047
:1045800002002000030028006400470010186900A2
:104590001090690070D4200010427800720520004D
:1045A0000240520005003A000200200003002800EB
:1045B000600047001018690010906900A270800028
:1045C000B3708000106F8000216F8000A31F070070
:1045D000361E07006007980020002000801F78002A
:1045E00060004700801F780068005700901F780027
:1045F000BE0B07006F00B10020002000801F780074
:1046000064004700801F780068005700901F780002
:10461000B60B07006F00B10010002000801F78006B
:104620006C004700801F780068005700901F7800DA
:10463000AE0B07006F00B1006A0057001000780051
:104640006007980010002000801F78006C00470071
:10465000801F780068004700801F7800A30B0700C8
:104660006F00B1000080FA00000006000000FA00B0
:104670006A005700901F780068005700901F78006C
:1046800080222F00801F780020E62000801F780005
:10469000AE1707008F00B10020E62000801F7800D1
:1046A000CF1707002F00B1000080FA0000000600BD
:1046B0000000FA006A005700901F78006800570059
:1046C000901F780050232F00801F780020E62000E4
:1046D000801F78009D1707008F00B10020E62000A2
:1046E000801F7800BE1707002F00B1000080FA007D
:1046F000000006000000FA0068005700901F7800D4
:104700006A005700901F780020242F00801F780037
:1047100020E62000801F78008C1707008F00B10072
:1047200020E62000801F7800AD1707002F00B100A1
:104730000080FA00000006009600FA0060004700C2
:1047400091482F00040009003158780065004700A7
:10475000E1482F0004000900315878006A00470042
:1047600031492F0004000900315878006F004700DC
:1047700081492F0004000900315878007400470077
:10478000D1492F000C000900315878001002200098
:1047900000004700A14A2F000B00090031587800A3
:1047A000D002200000004700614B2F0005000900E7
:1047B000315878003003200000004700C14B2F0023
:1047C00005000900315878009003200000004700E0
:1047D000214C2F000500090031587800F00320001B
:1047E00000004700814C2F00050009003158780077
:1047F0005004200000004700E14C2F000500090094
:1048000031587800B004200000004700414D2F00CF
:10481000040009003158780000052000000047001E
:10482000914D2F00040009003158780050052000F8
:1048300000004700E14D2F000500090031587800C5
:10484000B005200000004700414E2F000500090080
:10485000315878001006200000004700A14E2F00BC
:10486000040009003158780060062000000047006D
:10487000F14E2F0002000900315878009006200008
:1048800000004700214F2F00020009003158780036
:10489000C006200000004700514F2F000200090011
:1048A00031587800F006200000004700814F2F00AB
:1048B000020009003158780020072000000047005E
:1048C000B14F2F0002000900315878005007200036
:1048D00000004700E14F2F00020009003158780026
:1048E000800720000000470011502F00020009003F
:1048F00031587800B00720000000470041502F00D9
:104900000200090031587800E0072000000047004D
:1049100071502F0004000900315878003008200041
:1049200000004700C1502F000300090031587800F3
:10493000007580006B004000801F7800F0748000DC
:1049400061004000801F780048FF07004F00B10061
:1049500024708000600052000F003A003C0DF80007
:104960003E0DF800400DF800F0242F00801F780065
:1049700020E62000801F7800F4160700AF00B10089
:1049800020E62000801F7800151707002F00B100D7
:104990004E25040000000000E469800020E02000B3
:1049A0001002520044879800F069800050879800F8
:1049B000006A8000608798006000520008003D0097
:1049C000C4032000800820000000470010084200B7
:1049D00014002000A008200000004700100812006A
:1049E000A0082000000047001002780000E020002E
:1049F00010025200548798006000520008003D00E9
:104A0000C4032000A0082000000047001008420056
:104A100014002000C0082000000047001008120009
:104A2000C00820000000470010027800E0DF2000EE
:104A300010025200648798006000520004003D009C
:104A400084012000C0082000000047001008420038
:104A50008008200000004700901F7800A008200078
:104A600000004700901F7800C008200000004700A9
:104A7000901F780050262F00801F780020E620002D
:104A8000801F7800B1160700AF00B10020E62000BB
:104A9000801F7800D21607002F00B100007580003B
:104AA0006B004000801F780074172000E0E92000B0
:104AB00010005200801F7800ECFE07004F00B1008C
:104AC000107580000000E0000A0032004C0DF80074
:104AD0004E0DF80070272F00801F780020E6200080
:104AE000801F7800991607008F00B10094250400FC
:104AF00000000000606A8000716A8000A22121002D
:104B0000F3F12300801D0700801F7800811F7800CB
:104B100050282F00801F780020E62000801F78009A
:104B20008A1607008F00B10020E62000801F780061
:104B3000AB1607002F00B100340920000402470023
:104B4000400C2000004A78002475800035758000F4
:104B5000D0CC2C00C1D4230004017800850178005A
:104B6000F61D07000000E00002003C0000002000ED
:104B700001003700100020000000E00018003200A3
:104B80002475800035758000D0CC2C00C1D42B005A
:104B900004017800850178002B1E07000000E0006A
:104BA0000200350000002000010037001000200046
:104BB0000000E0000A00320024092000040247003F
:104BC000000A2000004A780034092000040247004F
:104BD000000C2000004A78001C26040000000000A1
:104BE0002075800031758000020020000300200045
:104BF000D21D07000000E00002003C000000200081
:104C000001003700100020000000E0000600320024
:104C1000240920000402470020082000004A7800F0
:104C20001C260400000000002409200004024700A4
:104C300010082000004A78004075800051758000FF
:104C400062708000737080002F1D0700A4708000C8
:104C5000B57080000401780085017800B71D070059
:104C60000000E00002003C000000200001003700CE
:104C7000100020000000E0000600320010042000B8
:104C8000801F7800751607002F00B1004C26040025
:104C900000000000801607000075800078004000CA
:104CA000801F780074172000E0E9200010005200F7
:104CB000801F78006DFE07004F00B1001075800066
:104CC0000000E0000A003200140EF800160EF80092
:104CD00030292F00801F780020E62000801F7800F8
:104CE0001A1607008F00B100922604000000000091
:104CF000A0708000B170800082942F001305240002
:104D0000011D0700801F7800811F7800F0292F0007
:104D1000801F780020E62000801F78000B16070017
:104D20008F00B10020E62000801F78002C160700BD
:104D30002F00B1005816070020092000000047008E
:104D4000104078000080FB00801F780030092000B0
:104D500000004700104078000080FB00801F7800B2
:104D6000C02A2F00801F780020E62000801F7800D6
:104D7000F61507008F00B100607580000000E000AC
:104D800014003A007475800085758000907580006D
:104D9000A17580000401780085017800671D070077
:104DA0000000E00002003C0000002000010037008D
:104DB000100020000000E000060032001004200077
:104DC000801F7800251607002F00B100EC26040094
:104DD00000000000301607000075800078004000D9
:104DE000801F7800F074800061004000801F780010
:104DF0001EFE07004F00B100AE0EF800B00EF80026
:104E0000502B2F00801F780020E62000801F7800A4
:104E1000CE1507008F00B10020E62000801F78002B
:104E2000EF1507002F00B1001B1607000403200038
:104E300020DD200010A2B900000D20000403400076
:104E400004EA2000E0082000000047001408530096
:104E5000F47480000009200000004700610842004F
:104E6000B4758000C57580000000200001F82300A3
:104E70000401780085017800731D07000000E00040
:104E80000200350000002000010037001000200063
:104E90000000E0006D003200E00820000000470044
:104EA000901F78000009200000004700901F780044
:104EB000EEFD07004F00B100B4758000C57580009D
:104EC000D0758000E17580000401780085017800CC
:104ED0001A1D07000000E00002003C000000200056
:104EE00001003700100020000000E0000600320042
:104EF00010042000801F7800D81507002F00B10093
:104F00008627040000000000E3150700B60EF80035
:104F1000B80EF800102C2F00801F780020E620002B
:104F2000801F7800891507008F00B10020E620005F
:104F3000801F7800AA1507002F00B100E0082000AC
:104F400000004700100078006D004000801F7800CE
:104F50000009200000004700901F7800C3FD0700F3
:104F60004F00B100BE0EF800C00EF800A02D2F00BB
:104F7000801F780020E62000801F7800731507004E
:104F80008F00B10020E62000801F780094150700F4
:104F90002F00B100E008200000004700100078005A
:104FA0007A004000801F78000009200000004700C0
:104FB000901F7800ADFD07004F00B100147680000F
:104FC00025768000307680004176800004017800EC
:104FD000850178001C1D07000000E000020035007C
:104FE0000000200001003700100020000000E00059
:104FF0000600320010042000801F7800971507007B
:105000002F00B1000828040000000000A2150700CE
:10501000C20EF800C40EF800602E2F00801F78002A
:1050200020E62000801F7800481507008F00B1009F
:1050300020E62000801F7800691507002F00B100CE
:10504000951507007628040000000000E008200005
:1050500000004700901F7800000920000000470072
:10506000901F780081FD07004F00B10060004700ED
:10507000801F78005A1507002F00B100E0082000BB
:1050800000004700100078006D004000801F78008D
:105090000009200000004700901F780073FD070002
:1050A0004F00B10065004700801F78004C150700D5
:1050B0002F00B100E0082000000047001000780039
:1050C0007A004000801F780000092000000047009F
:1050D000901F780065FD07004F00B1006A0047008F
:1050E000801F78003E1507002F00B100247080005B
:1050F00060005200C40132000403200020DD2000C3
:1051000010A2B900D00D20000402400000EA2000E7
:105110001000520070879800801F7800F41820005B
:10512000E0E9200010005200801F78004FFD0700CA
:105130004F00B10064708000757080005076800070
:105140006176800004017800850178007B1C0700EF
:105150000000E00002003C000000200001003700D9
:10516000100020000000E0002300320010758000D5
:105170000000E0000A0032000C0EF8000E0EF800ED
:10518000302F2F00801F780020E62000801F78003D
:10519000EE1407008F00B100F028040000000000AA
:1051A0006070800071708000A2212100F3F1230063
:1051B000D51B070002002000A3472400661D07003E
:1051C000801F7800811F7800E02F2F00801F78005B
:1051D00020E62000801F7800DC1407008F00B1005B
:1051E00020E62000801F7800FD1407002F00B1008A
:1051F00004290400000000006F004700801F7800B1
:10520000F71407002F00B100E0082000000047005D
:10521000100078006D004000801F7800B416200058
:10522000E0E9200010005200801F78000FFD070009
:105230004F00B10074004700801F7800E814070099
:105240002F00B1008470800095708000707680001F
:105250008176800004017800850178007A1C0700BF
:105260000000E000020035000000200001003700CF
:10527000100020000000E0000600320010042000B2
:10528000801F7800F51407002F00B1004C2904009E
:105290000000000000150700107580000000E0000D
:1052A0000A003200100EF800120EF800B0302F0085
:1052B000801F780020E62000801F7800A3140700DC
:1052C0008F00B1008629040000000000807080007B
:1052D00091708000A2212100F3F123008A1B0700B6
:1052E00002002000A34724001B1D0700801F780038
:1052F000811F780060312F00801F780020E6200099
:10530000801F7800911407008F00B10020E6200074
:10531000801F7800B21407002F00B100DE140700D0
:105320000403200020DD200010A2B900F0082000B6
:105330000403400004EA2000E008200000004700C9
:105340001408530036152000E4E92000000920006D
:105350000000470014085300646A8000756A8000EA
:105360000000200001F0230004017800850178008E
:10537000F21B07000000E00002003C0000002000DB
:1053800001003700100020000000E000CE003200D5
:10539000E008200000004700901F780084022000F1
:1053A000000920000000470010004200801F780024
:1053B000BFFC07004F00B1001002200000004700B2
:1053C000801F7800861407002F00B1001075800040
:1053D0000000E00040003200E0082000000047002C
:1053E000100078006D004000801F78000009200048
:1053F00000004700901F78009CFC07004F00B100A0
:10540000220EF800240EF80030322F00801F7800A2
:1054100020E62000801F78004C1407008F00B100A8
:1054200020E62000801F78006D1407002F00B100D7
:10543000E008200000004700100078007A004000DB
:10544000801F78000009200000004700901F7800AE
:1054500086FC07004F00B1002A0EF8002C0EF80061
:10546000F0332F00801F780020E62000801F780096
:10547000361407008F00B10020E62000801F78005E
:10548000571407002F00B10074022000E00820002C
:105490000000470010004200801F78000009200033
:1054A00000004700901F780070FC07004F00B1001B
:1054B000260EF800280EF80090352F00801F780087
:1054C00020E62000801F7800201407008F00B10024
:1054D0000C2B040000000000E00820000000470042
:1054E000100078006D004000801F78000009200047
:1054F00000004700901F78005CFC07004F00B100DF
:105500001071800021718000A2212100F3F123009D
:10551000FD1A0700801F7800811F780020372F00B8
:10552000801F780020E62000801F78000714070005
:105530008F00B10020E62000801F780028140700AB
:105540002F00B100E00820000000470010007800A4
:105550007A004000801F780000092000000047000A
:10556000901F780041FC07004F00B100507180008F
:105570006171800082942F0013052400E21A070055
:10558000801F7800811F7800E0382F00801F78008E
:1055900020E62000801F7800EC1307008F00B10088
:1055A00020E62000801F78000D1407002F00B100B6
:1055B00074022000E00820000000470010004200B4
:1055C000801F78000009200000004700901F78002D
:1055D00026FC07004F00B10030718000417180004F
:1055E000A2212100F3F12300C71A070002002000C6
:1055F000A3472400581C0700801F7800811F7800F3
:10560000903A2F00801F780020E62000801F78004D
:10561000CE1307008F00B10020E62000801F780025
:10562000EF1307002F00B100B4758000C57580002E
:105630000000200001F823000401780085017800B3
:10564000811B07000000E000020035000000200080
:1056500001003700100020000000E00016003200BA
:1056600044032000E0082000000047001000420032
:10567000801F78000009200000004700901F78007C
:10568000FAFB07004F00B100D20EF800D40EF8006C
:10569000403C2F00801F780020E62000801F78000B
:1056A000AA1307008F00B10020E62000801F7800B9
:1056B000CB1307002F00B10010002000B076880047
:1056C000042C040000000000B47680006100520049
:1056D0004D003A00E008200000004700901F7800CD
:1056E0008402200000092000000047001000420052
:1056F000801F7800EEFB07004F00B100D0022000B1
:1057000000004700801F7800B51307002F00B1008C
:10571000E008200000004700100078006D00400005
:10572000801F78000009200000004700901F7800CB
:10573000CEFB07004F00B1003003200000004700FF
:10574000801F7800A61307002F00B100E00820009A
:1057500000004700100078007A004000801F7800A9
:105760000009200000004700901F7800BFFB0700E1
:105770004F00B1009003200000004700801F780018
:10578000971307002F00B10074022000E0082000EA
:105790000000470010004200801F78000009200030
:1057A00000004700901F7800B0FB07004F00B100D9
:1057B000F003200000004700801F780088130700D6
:1057C0002F00B10044032000E00820000000470043
:1057D00010004200801F78000009200000004700F0
:1057E000901F7800A1FB07004F00B100500420007B
:1057F00000004700801F7800791307002F00B100D8
:1058000000002000B0768800247080006000520004
:105810001600320040758000517580006270800073
:1058200073708000381A0700A4708000B570800083
:105830000401780085017800C01A07000000E0002C
:1058400002003C0000002000010037001000200092
:105850000000E00005003A0064688000600052002B
:1058600002003200282D040000000000546880006F
:105870006000520076003A00007580006B00400026
:10588000801F780080072000801F780077FB0700CA
:105890004F00B100C46A80006300520009003D005F
:1058A000580DF800E03D2F00801F780020E6200012
:1058B000801F7800251307006F00B100702C0400D2
:1058C00000000000580DF800503F2F00801F7800A6
:1058D00020E62000801F78001C1307006F00B10035
:1058E00020E62000801F78003D1307002F00B10044
:1058F000007580006B004000801F7800600E200063
:10590000801F780059FB07004F00B10060D42000D1
:10591000104078000080FB00801F7800420DF800E6
:10592000440DF80020402F00801F780020E6200062
:10593000801F780005130700AF00B10020E62000AB
:10594000801F7800261307002F00B100007580002B
:1059500078004000801F7800600E2000801F7800D3
:1059600042FB07004F00B10070D4200010407800C7
:105970000080FB00801F7800480DF8004A0DF800F9
:1059800000412F00801F780020E62000801F780053
:10599000EE120700AF00B10020E62000801F780063
:1059A0000F1307002F00B100007580007800400041
:1059B000801F7800E0062000801F78002BFB070086
:1059C0004F00B100D06A8000E16A80000200200030
:1059D00003002000591A07000000E00002003C000C
:1059E0000000200001003700100020000000E0004F
:1059F0000E0032005A0DF8005C0DF800E0412F0057
:105A0000801F780020E62000801F7800CF1207005A
:105A10008F00B10020E62000801F7800F012070000
:105A20002F00B100202D040000000000B004200071
:105A300000004700801F7800E91207002F00B10026
:105A400010002000C0768800922D040000000000A5
:105A5000C47680006100520032003A000075800078
:105A60006B004000801F780080072000801F7800B6
:105A7000FEFA07004F00B1000005200000004700BB
:105A8000801F7800D61207002F00B100007580003B
:105A90006B004000801F7800600E2000801F78009F
:105AA000F2FA07004F00B100500520000000470047
:105AB000801F7800CA1207002F00B1000075800017
:105AC00078004000801F7800600E2000801F780062
:105AD000E6FA07004F00B100B005200000004700C3
:105AE000801F7800BE1207002F00B10000758000F3
:105AF00078004000801F7800E0062000801F7800BA
:105B0000DAFA07004F00B10010062000000047003D
:105B1000801F7800B21207002F00B10000002000A3
:105B2000C076880000002000408798000403200011
:105B300020DD200010A2B900900D200004034000D9
:105B400004EA2000E0082000000047001408530089
:105B5000C0082000008F9800806A8000916A800051
:105B6000D218070060879800C40620000402500085
:105B7000648798006000520004003D0084162000F5
:105B8000C00820000000470010084200C0082000A4
:105B90000000470010027800620020001100090098
:105BA0000202D80060879800640020000480B900D9
:105BB00060879800760220008408200004024700D5
:105BC0001400130090003D00C008200000004700B2
:105BD0001000780066034000668798008416200055
:105BE000040053000400350084162000C008200083
:105BF0000000470010081200C00820000000470005
:105C000010027800E2012000110009000202D80011
:105C100001007800600250000A00320040D92000E4
:105C2000860820000603470016024000D00220002C
:105C3000004A780010002000160B4000002F0400DE
:105C400000000000A4052000C0082000000047005C
:105C500010007800110009000400D800010078004D
:105C60006002500012003200C0082000000047000F
:105C7000901F780030432F00801F780044D9200007
:105C8000800820000000470010004200801F7800BC
:105C90002E1207006F00B1003400200080082000A1
:105CA0000000470010084200F82E04000000000029
:105CB00040D9200086082000060347001602400055
:105CC000D0022000004A780010002000160B40008F
:105CD000A82E040000000000240920000402470050
:105CE000E0042000004A7800D62E040000000000E6
:105CF000240920000402470050042000004A7800D4
:105D0000D62E0400000000002409200004024700F1
:105D100030052000004A7800D62E04000000000064
:105D2000240920000402470070052000004A780082
:105D3000D62E0400000000002409200004024700C1
:105D4000F0032000004A7800D62E04000000000076
:105D5000C0082000000047001002780060005200D8
:105D6000DDFF3200A6052000C40820000402470021
:105D700014001300DEFF3200460B2000C408200090
:105D80000402470014001300DFFF3200C0082000A7
:105D90000000470010037800E410200004005300C6
:105DA000DFFF32009C2E04000000000040D92000DC
:105DB0008608200006034700160240002009200044
:105DC00000004700104A78000600780010007800B4
:105DD000610240004487980040D92000040240003E
:105DE000D0022000004A780010002000160B40006E
:105DF000C4002000C0082000000047001008420036
:105E0000DA2D04000000000044D9200080082000A2
:105E1000000047001002420000002000004A780005
:105E2000806A8000916A80002018070040879800EF
:105E300064002000110009000400D800010078006F
:105E4000408798006002500005003A0064DB2000A3
:105E500000002000004A7800362F040000000000F7
:105E600074DB200000002000004A780000092000B8
:105E70000000470010027800800820000000470062
:105E8000100352004687980074DB200000002000B9
:105E9000004A7800E0082000000047001000780069
:105EA0006A004000801F7800861F780000FA070013
:105EB0004F00B10070D92000801F780080432F0070
:105EC000801F780020E62000801F78009F110700C7
:105ED0006F00B10020E62000801F7800C01107008D
:105EE0002F00B100C4708000D5708000826A8000ED
:105EF000936A800004007800850078001419070078
:105F0000EA17070060879800E008200000004700BB
:105F1000901F7800A4052000000920000000470021
:105F200010004200801F7800E1F907004F00B10027
:105F3000C0082000000047001002780060005200F6
:105F40000D003A00207080000000E0000A003200DE
:105F5000500DF800520DF800D0432F00801F78003C
:105F600020E62000801F7800781107008F00B10024
:105F7000CC2F040000000000500DF800520DF80076
:105F800090442F00801F780020E62000801F7800BA
:105F90006E1107008F00B10020E62000801F7800FE
:105FA0008F1107002F00B100BB1107002070800087
:105FB0000000E00027013200C00820000000470078
:105FC000100278006000520004003D00841620009A
:105FD000C00820000000470010084200460B2000C7
:105FE000C408200004024700140013000400340019
:105FF00084162000C008200000004700100812008E
:106000000000200050879800A008200000004700F2
:10601000100278007F0052000C003D0044D920009F
:10602000A0082000000047001002420000022000EB
:10603000004A780014002000A0082000000047005B
:1060400010084200043004000000000044D9200081
:10605000A0082000000047001002420000002000BD
:10606000004A780006FA2F00C40820000402470006
:10607000140013002400340006062000C408200089
:1060800004024700140013001F003D00A405200077
:10609000C00820000000470010024200248F980032
:1060A0005487980062002000110009000202D80005
:1060B0000100780040879800640020002E8890003E
:1060C000110009000400D8005087980060025000B9
:1060D0000B003500A00820000000470010027800E7
:1060E0007F00520006003D0044D92000A008200097
:1060F000000047001002420080042000004A78009F
:106100008830040000000000000020004087980054
:1061100080082000000047001002780000092000DD
:10612000000047001002420044879800E008200069
:10613000000047001000780074004000801F7800C5
:10614000841F78005AF907004F00B100C0082000F2
:106150000000470010027800600052000A003A0078
:1061600040D92000801F780000452F00801F780054
:1061700020E62000801F7800F41007006F00B100B7
:106180000031040000000000C008200000004700AB
:1061900010027800670052000700350096FF2F00BC
:1061A000C4082000040247001400130002003C0051
:1061B000F03004000000000040D92000801F78006B
:1061C000F0452F00801F780020E62000801F780017
:1061D000DE1007006F00B100003104000000000075
:1061E00040D92000801F780040462F00801F780093
:1061F00020E62000801F7800D41007006F00B10057
:1062000020E62000801F7800F51007002F00B10065
:10621000C008200000004700100278006000520013
:1062200024003A00E0082000000047001000780039
:106230006A004000801F780000092000000047002D
:106240001000780067005000801F780007F90700F1
:106250004F00B1006006200000004700801F78005A
:10626000DF1007002F00B100E00820000000470009
:10627000100078006A004000801F7800F40B2000B6
:10628000000920000000470010004200801F780035
:10629000F6F807004F00B10090062000000047000C
:1062A000801F7800CE1007002F00B10026320400B6
:1062B00000000000C0082000000047001002780025
:1062C000600052002E003D00E00820000000470062
:1062D000100078006A004000801F7800000920004C
:1062E000000047001000780067005000801F780011
:1062F000DEF807004F00B10066FA2F00C408200046
:10630000040247001400130007003D00C0062000EF
:1063100000004700801F7800B11007002F00B10077
:106320009E31040000000000F0062000000047003D
:10633000801F7800AA1007002F00B100E00820009D
:1063400000004700100078006A004000801F7800BD
:10635000F40B20000009200000004700100042005C
:10636000801F7800C1F807004F00B100200720000F
:1063700000004700801F7800991007002F00B1002F
:10638000C0082000000047001002780060005200A2
:106390002E003400E00820000000470010007800C4
:1063A0006A004000801F7800F40B200000092000E4
:1063B0000000470010004200801F7800ABF8070083
:1063C0004F00B100A6052000C408200004024700C9
:1063D000140013000700340050072000000047009D
:1063E000801F78007E1007002F00B10004320400E7
:1063F000000000008007200000004700801F780098
:10640000771007002F00B100E008200000004700CF
:10641000100078006A004000801F7800000920000A
:10642000000047001000780067005000801F7800CF
:106430008EF807004F00B100B007200000004700B1
:10644000801F7800661007002F00B100CE330400D3
:1064500000000000106B80000000E000CF00320060
:10646000906E80006B02400074879800000020004E
:10647000106B8800841F7800B0002000801F780017
:106480009CF807004F00B1000000200040879800F2
:106490008008200000004700100278006C005200C5
:1064A0003E003D00800820000000470010007800FA
:1064B0004202DD0040D6200004004000620340009C
:1064C00024032000160012000600310034092000C9
:1064D0000402470000092000004A7800A4320400AA
:1064E0000000000080082000000047001000780035
:1064F0004202DD0040D6200004004000620240005D
:106500001003200014021000720020001100090086
:106510000282D80004092000000242003009200055
:106520000000470004487800044378006409200014
:1065300004405300040036003409200004024700E0
:1065400060092000004A7800300920000000470060
:10655000104078000080FB00801F780090462F00DC
:10656000801F780020E62000801F7800F70F0700CA
:106570006F00B10020E62000801F7800181007008F
:106580002F00B10014002000800820000000470008
:10659000100842004832040000000000E00820001B
:1065A000000047001000780061004000801F780064
:1065B000B0002000801F78004EF807004F00B100A7
:1065C000000020004087980080082000000047005D
:1065D000100278006C00520034003D00800820005A
:1065E00000004700100078004202DD0040D6200085
:1065F0000400400062034000140320001600120053
:106600000600390034092000040247006009200018
:10661000004A78002C3304000000000080082000AD
:1066200000004700100078004202DD0040D6200044
:106630000400400062004000100278007200200058
:10664000110009000282D800060920003409200048
:1066500004024700004A43003009200000004700C0
:10666000104078000080FB00801F780060472F00FA
:10667000801F780020E62000801F7800B30F0700FD
:106680006F00B10020E62000801F7800D40F0700C3
:106690002F00B100140020008008200000004700F7
:1066A00010084200E432040000000000E00820006E
:1066B000000047001000780062004000801F780052
:1066C000B0002000801F78000AF807004F00B100DA
:1066D000E007200000004700801F7800C00F07007F
:1066E0002F00B100000020004087980080082000A3
:1066F00000004700100278006C00520027003D00A7
:106700008008200000004700100078004202DD00F1
:1067100040D62000040040001002780060005200C3
:1067200013003200800820000000470010007800AD
:106730004202DD0040D6200004004000901F780097
:1067400030482F00801F780020E62000801F78004E
:106750007E0F07006F00B10020E62000801F780048
:106760009F0F07002F00B100C2330400000000009B
:106770003008200000004700801F7800980F0700B5
:106780002F00B10014002000800820000000470006
:106790001008420076330400000000000080FA0078
:1067A000000006000600FA006000470001512F00BB
:1067B000040009003158780060004700801F78000D
:1067C000870F07002F00B1000080FA0000000600CC
:1067D0000600FA0080012000000F7800926E800011
:1067E000300020000090B900F0014000230798001D
:1067F00068015700120078001007980012801100FD
:1068000007003400C00D2000000F7800640047002E
:10681000100078006101400062004700100811007C
:106820006200470010017800D00020000090B900FD
:10683000100798007A00400010079800801F780029
:1068400060004700901F780050512F00801F780093
:1068500020E62000801F78003C0F07008F00B10069
:1068600020E62000801F78005D0F07002F00B10098
:106870000080FA00000006004200FA0060004700B5
:10688000217A2F0003000900315878006400470086
:10689000617A2F0003000900315878006800470032
:1068A000A17A2F0003000900315878006C004700DE
:1068B000E17A2F000300090031587800700047008A
:1068C000217B2F000600090031587800770047002F
:1068D000917B2F0008000900315878000002200049
:1068E00000004700217C2F00030009003158780088
:1068F0004002200000004700617C2F0004000900D6
:10690000315878009002200000004700B17C2F0031
:106910000300090031587800D00220000000470031
:10692000F17C2F0005000900315878003003200069
:1069300000004700517D2F00030009003158780006
:106940007003200000004700917D2F000300090024
:1069500031587800B003200000004700D17D2F009F
:106960000100090031587800D003200000004700E2
:10697000F17D2F00040009003158780068005700AD
:10698000901F780092FF07002F00B10068005700A9
:1069900010017800A1ED20001100510006003A001E
:1069A000A0042000801F78002C0F07002F00B100EA
:1069B000DE34040000000000370F07009C3704009D
:1069C00000000000CE0EF800D00EF80020522F007C
:1069D000801F780020E62000801F7800DB0E070073
:1069E0008F00B1008038040000000000A80EF800FD
:1069F000AA0EF800A0532F00801F780020E6200088
:106A0000801F7800D10E07008F00B100803804008D
:106A100000000000080EF8000A0EF80020552F00B4
:106A2000801F780020E62000801F7800C70E070036
:106A30008F00B1008038040000000000060EF8004E
:106A4000A0562F00801F780020E62000801F7800CD
:106A5000BE0E07006F00B100803804000000000087
:106A6000CA0EF800CC0EF80000582F00801F7800E6
:106A700020E62000801F7800B40E07008F00B100D0
:106A80008038040000000000400EF800420EF800BC
:106A900080592F00801F780020E62000801F78009A
:106AA000AA0E07008F00B10080380400000000002B
:106AB000DC0EF800DE0EF800005B2F00801F78006F
:106AC00020E62000801F7800A00E07008F00B10094
:106AD00080380400000000003C0EF8003E0EF80074
:106AE000805C2F00801F780020E62000801F780047
:106AF000960E07008F00B1008038040000000000EF
:106B0000E00EF800E20EF800005E2F00801F780013
:106B100020E62000801F78008C0E07008F00B10057
:106B20008038040000000000E40EF800E60EF800D3
:106B3000805F2F00801F780020E62000801F7800F3
:106B4000820E07008F00B1008038040000000000B2
:106B5000480EF8004A0EF80000612F00801F7800F0
:106B600020E62000801F7800780E07008F00B1001B
:106B70008038040000000000440EF800460EF800C3
:106B800080622F00801F780020E62000801F7800A0
:106B90006E0E07008F00B100803804000000000076
:106BA000340EF800360EF80000642F00801F7800C5
:106BB00020E62000801F7800640E07008F00B100DF
:106BC0008038040000000000380EF8003A0EF8008B
:106BD00080652F00801F780020E62000801F78004D
:106BE0005A0E07008F00B10080380400000000003A
:106BF000E80EF800EA0EF80000672F00801F78000A
:106C000020E62000801F7800500E07008F00B100A2
:106C10008038040000000000C60EF800C80EF8001E
:106C200080682F00801F780020E62000801F7800F9
:106C3000460E07008F00B1008038040000000000FD
:106C4000D17280006180500004003A00600047006B
:106C50008000780032360400000000006400470025
:106C60008000780001007800801F7800006A2F0003
:106C7000801F780020E62000801F7800330E070078
:106C80006F00B1008038040000000000F172800045
:106C90006180500004003A006800470080007800DE
:106CA00058360400000000006C00470080007800A7
:106CB00001007800801F7800606B2F00801F780033
:106CC00020E62000801F7800200E07006F00B10032
:106CD0008038040000000000107580000000E00013
:106CE0000400320070004700800078007E36040007
:106CF0000000000077004700800078000100780065
:106D0000801F7800C06C2F00801F780020E62000D4
:106D1000801F78000D0E07006F00B100803804005E
:106D200000000000200DF800F06D2F00801F78009B
:106D300020E62000801F7800040E07006F00B100DD
:106D40008038040000000000906E80000000E00029
:106D5000050032000002200000004700800078009B
:106D6000BA36040000000000400220000000470086
:106D70008000780001007800801F7800506F2F009D
:106D8000801F780020E62000801F7800EF0D0700AC
:106D90006F00B1008038040000000000EC0EF80025
:106DA00080702F00801F780020E62000801F780070
:106DB000E60D07006F00B1008038040000000000FD
:106DC000207080000000E0000500320090022000EA
:106DD0000000470080007800F63604000000000044
:106DE000D0022000000047008000780001007800F9
:106DF000801F7800E0712F00801F780020E62000BF
:106E0000801F7800D10D07006F00B10080380400AA
:106E100000000000EE0EF800F00EF80010732F00D6
:106E2000801F780020E62000801F7800C70D070033
:106E30008F00B1008038040000000000F20EF8005E
:106E4000F40EF80080742F00801F780020E62000E8
:106E5000801F7800BD0D07008F00B100803804004E
:106E6000000000009E0EF80000762F00801F7800C2
:106E700020E62000801F7800B40D07006F00B100ED
:106E80008038040000000000607580000000E00011
:106E90000500320030032000000047008000780029
:106EA0005A37040000000000700320000000470073
:106EB0008000780001007800801F780060772F0044
:106EC000801F780020E62000801F78009F0D0700BB
:106ED0006F00B1008038040000000000B07780002F
:106EE0000000E00005003200B00320000000470071
:106EF000800078008437040000000000D0032000E8
:106F0000000047008000780001007800801F7800B2
:106F1000C0782F00801F780020E62000801F7800B6
:106F20008A0D07006F00B1008038040000000000E7
:106F300080380400000000006800570090007800CE
:106F4000608050009FFE320068005700900078007B
:106F500061805000A5FE3200680057009000780064
:106F600062805000ABFE320068005700900078004D
:106F700063805000B1FE3200680057009000780036
:106F800064805000B6FE3200680057009000780020
:106F900065805000BCFE3200680057009000780009
:106FA00066805000C2FE32006800570090007800F2
:106FB00067805000C8FE32006800570090007800DB
:106FC00068805000CEFE32006800570090007800C4
:106FD00069805000D4FE32006800570090007800AD
:106FE0006A805000DAFE3200680057009000780096
:106FF0006B805000E0FE320068005700900078007F
:107000006C805000E6FE3200680057009000780067
:107010006D805000ECFE3200680057009000780050
:107020006E805000F2FE3200680057009000780039
:107030006F805000F8FE3200680057009000780022
:1070400070805000FEFE320068005700900078000B
:10705000718050000DFF32006800570090007800EA
:10706000728050001CFF32006800570090007800CA
:10707000738050002BFF32006800570090007800AA
:107080007480500030FF3200680057009000780094
:107090007580500041FF3200680057009000780072
:1070A0007680500046FF320068005700900078005C
:1070B0007780500057FF320068005700900078003A
:1070C000788050005DFF3200680057009000780023
:1070D0007980500063FF320068005700900078000C
:1070E0007A80500068FF32006800570090007800F6
:1070F0007B80500079FF32009837040000000000C8
:1071000020E62000801F7800350D07002F00B10019
:107110000080FA00000006000200FA0000002000D3
:10712000000F780060004700900078007B805000DE
:1071300009003C0060004700901F7800CEFD07006A
:107140002F00B100110020006000470010884000AF
:1071500092380400000000000080FA0000000600E1
:107160000000FA00A2072000E800570011001100FB
:1071700007003E0012062000E80057001100110031
:1071800003003900F1FD2F006800570010886000EF
:107190004EB897000080FA00000006000200FA00D6
:1071A00000002000000F7800680057009000780071
:1071B00060004700108040009040780060C05000A0
:1071C0001300320071108000002020000080600059
:1071D000C900DE000100E00002003200E2380400D5
:1071E00000000000680057001000780060014700B0
:1071F00092004000114078000080FB008010880061
:107200001000200012094000D438040000000000E3
:107210000080FA00000006000C00FA0020002000A8
:10722000000F780000002000300798006800570029
:107230009000780066004700108040009040780081
:1072400060C050000C003200680057001000780049
:107250006601470012004000904078008180FB00EA
:1072600060004700108868001000200012094000EC
:10727000163904000000000060004700901F7800ED
:10728000407E2F00801F780062004700801F78003A
:10729000AE0C07006F00B10000002000300798001E
:1072A000E2004700660047001080400090407800F0
:1072B00060C0500011003200E20047006600470045
:1072C0005007980010804000400798001040780058
:1072D0000080FB00801F7800A1FF07002F00B10095
:1072E000CE00900080487800110020005E009000E1
:1072F0001088400050390400000000006200470080
:10730000801F780068005700901F7800907E2F0043
:10731000801F780040D92000801F78008B0C070068
:107320008F00B10040D92000801F78009BFF07002C
:107330002F00B1000080FA00000006002A00FA00C9
:1073400060004700617F2F000E000900315878006F
:107350006F00470051802F0001000900315878006C
:107360007100470071802F0001000900315878003A
:107370007300470091802F001600090031587800F3
:1073800060004700801F7800A3FF07002F00B100B6
:107390004EB897000000E000060032006F00470082
:1073A000801F78009CFF07002F00B100E239040025
:1073B0000000000071004700801F780096FF070062
:1073C0002F00B10073004700801F780092FF070074
:1073D0002F00B1000080FA00000006000000FA0053
:1073E000EA00570011007800103B880062804000DE
:1073F0009040780020032000014878006C0057007E
:1074000010007800003B88000C0007000080FA00A4
:10741000000006000000FA0040042400801F7800ED
:107420006A005700B01F7800A01F7800EBFF07002C
:107430006F00B1000080FA00000006000000FA00B2
:107440000500FC005C0520003C3B8800AC0A2000E5
:107450003C3B880061E7A80000000000000000003D
:107460000080FA00000006000000FA006A005700E1
:10747000B01F7800A01F7800E6FF07004F00B100A2
:10748000013B80000000280000806000CF00DE008B
:107490000100E00002003200403A04000000000059
:1074A000EA00570011007800C000880062804000A8
:1074B0009040780020032000014878006C005700BD
:1074C00010007800B00088000B0EBB0040002400C4
:1074D000003B8800D9FF0700F1FF2B000076200059
:1074E000108860000080FA00000006000A00FA0020
:1074F0006A00570010007800100798004EB99700F6
:1075000032007800A2007800200798003107980028
:1075100000002000000F7800600047001002780093
:107520006C015700120052001D003D001E0090002B
:10753000901F78006400470040079800B01F780053
:10754000A01F7800C8FF07006F00B10022002000D4
:10755000620047001008410022002000CF91DE00A9
:107560004E0090001018410010904900023B80002E
:1075700000002800000061004F01DE000200E00072
:1075800002003200B63A04000000000012002000A1
:1075900060004700100841008C3A04000000000021
:1075A0006C005700100078004100DD004EB99700D4
:1075B000CF80DE0012194000129148000080FA00CE
:1075C000000006000000FA0092032000E8005700C7
:1075D0001100110008003E0002032000E8005700DF
:1075E00011001100040039001000200080407800D4
:1075F000003B0400000000000000200080407800F4
:107600008180FB00010078000080FA000000060085
:107610000600FA00680057001042780060405200EF
:1076200072003D0068025700144078000000FB0023
:1076300060001000004A780000437800E406200053
:10764000044053003A0035006800570020079800B6
:10765000104278000402FB00420620000402FB00F6
:10766000110009000202D800720040004202DD0051
:1076700000822F000400400030027800A002780051
:107680002E0090000407980015079800104278001B
:107690000402FB0042062000110009000202D8008B
:1076A00001007800A4002000110009000400D800A7
:1076B000690040004202DD0000822F00040040000B
:1076C00030027800A00278000E0090009E0090002A
:1076D00004017800850178008B1207002E029000CB
:1076E0000007980011079800040078001042780005
:1076F0000402FB00A2002000110009000202D800D1
:10770000010078004202DD0000822F0004004000EA
:1077100030027800A00278000E0090009E009000D9
:107720000401780085017800771207009C0037007B
:1077300068005700104278006A405200220034006E
:107740006800570000079800104278000402FB0010
:10775000A20020000402FB00110009000202D80070
:10776000690040004202DD0000822F00040040005A
:1077700030027800A00278000E0090000407980004
:1077800015079800104278000402FB00A2002000B8
:10779000110009000202D800010078004202DD0059
:1077A00000822F000400400030027800A002780020
:1077B0000E0090009E009000040178008501780082
:1077C000511207007600370068005700104078001B
:1077D0000000FB004202DD0000822F000402400096
:1077E00034007800A40078006D003700680057006E
:1077F00010437800E4062000044053003A003500AE
:107800006800570020079800104278000402FB002F
:10781000420620000402FB00110009000202D80009
:10782000720040004202DD0040852F00040040004D
:1078300030027800A00278002E0090000407980023
:1078400015079800104278000402FB004206200051
:10785000110009000202D80001007800A4002000F5
:10786000110009000400D800690040004202DD0058
:1078700040852F000400400030027800A00278000C
:107880000E0090009E0090000401780085017800B1
:107890001D1207002E0290000007980011079800A3
:1078A00004007800104278000402FB00A2002000CF
:1078B000110009000202D800010078004202DD0038
:1078C00040852F000400400030027800A0027800BC
:1078D0000E0090009E009000040178008501780061
:1078E000091207002E003700680057001042780088
:1078F0006A405200220034006800570000079800D8
:10790000104278000402FB00A20020000402FB00E9
:10791000110009000202D800690040004202DD00A7
:1079200040852F000400400030027800A00278005B
:107930000E00900004079800150798001042780088
:107940000402FB00A2002000110009000202D8007E
:10795000010078004202DD0040852F000400400055
:1079600030027800A00278000E0090009E00900087
:107970000401780085017800E31107000800370052
:1079800068005700104078000000FB004202DD0054
:1079900040852F000402400034007800A4007800E5
:1079A0000080FA00000006000600FA006800570098
:1079B00010437800E4062000044053003E003900E4
:1079C0006800570020079800104278000482FB00EE
:1079D000420620000402FB00110009000202D80048
:1079E000720040004202DD0000822F0004024000CD
:1079F00034007800A40078000200200003F0230087
:107A0000C11107002E02900000079800110798008E
:107A100004007800104278000482FB004206200037
:107A2000110009000202D80001007800A400200023
:107A3000110009000400D800690040004202DD0086
:107A400000822F000400400030027800A00278007D
:107A50000E0090009E0090000401780085017800DF
:107A6000A91107002E029000000798001107980046
:107A700004007800104278000482FB00A20020007D
:107A8000110009000202D800010078004202DD0066
:107A900000822F000400400030027800A00278002D
:107AA0000E0090009E00900004017800850178008F
:107AB0009511070035003700680057001042780024
:107AC0006A40520026003600680057000007980000
:107AD000104278000482FB00A20020000402FB0098
:107AE000110009000202D800690040004202DD00D6
:107AF00000822F000402400034007800A4007800C7
:107B00000200200003F023007F1107000E02900006
:107B100000079800110798000400780010427800D0
:107B20000482FB00A2002000110009000202D8001C
:107B3000010078004202DD0000822F0004004000B6
:107B400030027800A00278000E0090009E009000A5
:107B500004017800850178006B1107000B003700E5
:107B600068005700104078000080FB004202DD00F2
:107B700000822F000402400034007800A400780046
:107B80000200200003F023005F1107000080FA00CC
:107B9000000006000000FA0002000700323E040068
:107BA000000000000001BE00190007000470A700DB
:107BB00003F0A10003F8A30013003A006509B10027
:107BC00010003200090035006928E100020035008C
:107BD00001002800000005000000400081804800EE
:107BE0008502E900FCFF3A0000000600F88F420021
:107BF000050035008100D1000080D3008502E80037
:107C0000FCFF3A00000006008000EB0000000500C9
:107C1000C70ADE00F107B200F50FB200080032001B
:107C2000E1CF4200020032000170A00024000500F4
:107C3000810F7000010032000408050044000500B7
:107C4000810F700002003A00140005008502E9006F
:107C50000000400081C04800FCFF3B000170A00014
:107C6000240005000080FA00000006000000FA0071
:107C7000020007008A3E0400000000000400E0004B
:107C800002003A001000070000000600811F780083
:107C90000100E00002003D0060001000E0801800DC
:107CA0000300E00002003D0060011100E0811900C6
:107CB000050007004F00E00002003B0060001000DC
:107CC000E080180000000600020007000400BE006B
:107CD000000006006022B800060220000000D0006C
:107CE0008180D2000482D2008582D2000000A000F0
:107CF0000202520083825A0003003B00020242004B
:107D000083824A000000A1000603E900F3FF3A0065
:107D1000000006000080FA00000006000000FA00E3
:107D200002000700DC3E0400000000000400E00048
:107D300002003A001000070000000600839F680060
:107D40000100E00002003D0060001000E08018002B
:107D50000300E00002003D0060011100E081190015
:107D6000050007004F00E00002003B00600010002B
:107D7000E0801800000006006022B8000602200023
:107D80000000D0008180D2000482D2008582D2001F
:107D90000000A0000202520083825A0003003B0050
:107DA0000202420083824A000000A1000603E900AB
:107DB000F3FF3A00000006000080FA000000060011
:107DC0002800FA006000470021922F0006000900F9
:107DD0003158780000002000000F980000002000BB
:107DE000700798003EBB9700140020006A005700FF
:107DF00010084200164278006A00470004487800E4
:107E00000404E000CE0932006A0047001043780005
:107E100054022000044053000B0032006A02470065
:107E20004EB89700144878001400200068005700EE
:107E300010084200140020007000470010084200A3
:107E4000F23E0400000000000000200060079800DF
:107E50000000200070079800803F04000000000030
:107E6000840020006E0047001008720014002000FB
:107E70006A00570010084200B63F040000000000EE
:107E8000140020006E00470010087200140020004B
:107E90006A00570010084200B63F040000000000CE
:107EA000240020006E00470010087200140020001B
:107EB0006A00570010084200B63F040000000000AE
:107EC000048020006E00470010087200140020009B
:107ED0006A00570010084200B63F0400000000008E
:107EE000440020006E0047001008720014002000BB
:107EF0006A00570010084200B63F0400000000006E
:107F00003EB8970010437800D4022000044053008C
:107F1000D3FF32003EB897001043780004022000DF
:107F200004405300D6FF32003EB89700104378005B
:107F3000B402200004405300D9FF32003EB897003D
:107F4000104378003402200004405300DCFF32006C
:107F50003EB897001043780004032000044053000B
:107F6000DFFF3200BA3F0400000000002C3F040095
:107F7000000000006E004700100078006202600000
:107F800003003200E4FF2F006E004700100862007B
:107F90006E004700100078006802600003003200A5
:107FA000B4FF2F006E004700100862003EB8970033
:107FB000104078000080FB00801F780081FD0700E2
:107FC0002F00B1000000E000190032000000200086
:107FD000600798006C03470016027800A00020009C
:107FE00000A2B9003EB89700104078000080FB0066
:107FF0000002420000032000000B52006A005700FC
:10800000100078006100400030BF9F0010407800F1
:108010000080FB00801F78006AFD07002F00B10080
:108020000000E000EBFF3A003640040000000000D2
:108030003EB8970010437800A4022000044053008B
:108040000A003A002EBB97002EBA970020002000AD
:10805000140A1000160278001400780060079800D7
:10806000140020006A005700100842003EB8970034
:1080700010437800E4022000044053002F003A002F
:108080006A005700100078006100400030BF9F0078
:1080900010437800A4022000044053000C003A0072
:1080A0002EBB97002EBA970020002000140A100063
:1080B0001602780014007800400798001400200091
:1080C0006A005700100842009A40040000000000B7
:1080D00000002000400798003EB89700104078004C
:1080E0000080FB00801F780036FD07002F00B100E4
:1080F0000000E0000F00320068034700160278001D
:10810000A000200000A2B9003EB8970010407800FF
:108110000080FB000002420000032000000B520020
:10812000140020006A005700100842006C40040050
:1081300000000000A8400400000000000000200033
:1081400040079800040021006E00470010087200EC
:108150003EBB9700140020006A0057001008420040
:10816000164278006A004700044878002E42040056
:10817000000000000E089000F20837000401200003
:108180006E00470010087200A840040000000000C4
:10819000044020006E00470010087200D042040026
:1081A00000000000040220006E004700100872006A
:1081B000041020006E00470010087200D042040036
:1081C00000000000042020006E004700100872002C
:1081D000D042040000000000040420006E004700AC
:1081E00010087200D042040000000000D0420400D9
:1081F00000000000040220006E004700100872001A
:10820000040820006E00470010087200D0420400ED
:1082100000000000F8044700090478002EBB970016
:108220002EBA970020002000140A100016007800D3
:10823000100C7800190278006000520003003A0028
:108240007802470060004700000A78007800470085
:108250006202400000002000000A78007803470016
:108260006202430016007800140240001404E0008B
:1082700006003200780047006202400014007800D7
:10828000610A40002E410400000000004E009000F2
:108290000000E0000B00320078004700620340005D
:1082A00068004700100278001600520005003100F7
:1082B0007800470062024000680047001000780024
:1082C000000A780078004700620340006C00470015
:1082D00010027800160052000700360078004700B0
:1082E00062004000100278006C0047001008120085
:1082F000804104000000000000002000600798009A
:108300006E004700100078006802600011003A001B
:108310006E039000140020006C004700100812004B
:108320000600E0000B0032004EBA97000002200069
:10833000004A78001400200068005700100842002E
:10834000140020007000470010084200884104001B
:108350000000000078004700620340001602780029
:1083600016007800610B50000400E0000F0032009E
:108370007800470000037800100278004EB897009C
:1083800014487800140020006800570010084200CC
:1083900016007800610B40001400200070004700B8
:1083A00010084200AA410400000000006E004700CF
:1083B0001000780068026000110032006E03900027
:1083C000140020006C004700100812000600E000B6
:1083D0000B0032004EBA970000022000004A7800DD
:1083E000140020006800570010084200140020000C
:1083F0007000470010084200DE4104000000000049
:10840000F23E0400000000002EBB97002EBA970039
:1084100020002000140A1000160078001042780096
:108420006A00470004487800780247006A00470065
:10843000000A78006202420010002000000A780062
:108440004641040000000000040C20006E004700BC
:1084500010087200D0420400000000006A004700CB
:10846000104278006040520042FF32006A0047002C
:1084700010437800C4042000044053003FFF320042
:108480006A00470010437800C406200004405300EF
:108490003AFF32006A00470010437800640620006B
:1084A000044053003AFF32006A004700104378004E
:1084B00054042000044053003AFF32006A00470091
:1084C00010437800540620000440530038FF320067
:1084D0006A004700104378007406200004405300EF
:1084E00038FF32006A00470010437800F40620008D
:1084F0000440530038FF32006A0047001043780000
:10850000440620000440530038FF32006A00470050
:1085100010437800940620000440530033FF3200DB
:108520006A0047001043780004072000044053000D
:1085300030FF32006A0047001043780084052000B5
:10854000044053002BFF32006A00470010437800BC
:10855000840720000440530029FF32006A004700CE
:1085600010437800340720000440530029FF3200F4
:108570006A0047001043780034062000044053008E
:10858000A1FF32006A004700104378005407200022
:1085900004405300ACFF320014420400000000000D
:1085A0006E00470010027800007020000002620098
:1085B0005F0532006E0047001002780000002100C5
:1085C00000026200020032006000200040079800B4
:1085D0002EBB97002EBA970040002000140A10000E
:1085E0001602780034007800A4007800100F98007C
:1085F000210F98000200200003002000920F0700C6
:108600000000E000020035000000200001003700FB
:10861000100020000000E0000800320004002000EC
:10862000050028007200470010186A0010906A00C8
:10863000340020006E004700100872000000200087
:10864000300F98007202470034007800A4007800D0
:1086500002002000030020007B0F07000000E00064
:1086600002003A0000002000010037001000200046
:108670000000E00058003200760447007203470013
:1086800070012000CF80DE0036027800A60278005C
:108690000000E900030035008502D1000482D30008
:1086A000FBFF3700F00F200000026200E00720000F
:1086B000000C5200080078001000780061025000A1
:1086C000340F98003000200000A2B900340F980049
:1086D000A2002000110009000202D800300F98000B
:1086E0006002500003003D001400200076004700A7
:1086F000100812007800470000179800600F9800DB
:10870000760047001000780060001000801F78009D
:10871000BFFB07002F00B1001E099000AE099000BA
:10872000790E07006E0A9000001A78000112780096
:108730000E12900034007800A40078000002780047
:10874000810278000000200001F823000401780075
:1087500085017800F90E07000000E00002003C00EF
:108760000000200001003700100020000000E000A1
:1087700005003200140020007600470010081200A7
:10878000EC43040000000000780247003400780049
:10879000A400780000027800810278000000200028
:1087A000011224000401780085017800260F0700DB
:1087B0000000E0000200340000002000010037004B
:1087C000100020000000E000030032001400200030
:1087D000760047001008420076004700100278003B
:1087E0006000520005003C006A02470010002000B3
:1087F000004A780006440400000000006A024700B6
:108800007600470010407800004A78006E0047006C
:1088100010027800001020000002620014003A00EC
:108820006E00470010027800002020000002620065
:108830000D003200C6FF2F0076024700140013001F
:1088400007003500760047001003780068024700F3
:108850001400530002003D003444040000000000F6
:108860003844040000000000DC4804000000000060
:108870004E0090000000E000080032006E0047004B
:108880001002780000202000000262000300320085
:10889000140020006800470010081200680047001C
:1088A0001002780068005200050036006A02470096
:1088B00080002000004A78006844040000000000A6
:1088C0006A0247006800470010407800004A7800BC
:1088D0007202470034007800A400780002002000F3
:1088E00003002000D80E07000000E00002003A005C
:1088F0000000200001003700100020000000E00010
:10890000700032007600470010007800801F780069
:108910003FFB07002F00B1000001780081017800C3
:108920001E089000AE0890008B0F0700100F9800F3
:10893000210F98006A004700104078000080FB007B
:1089400060001000801F780031FB07002F00B1008D
:1089500000017800810178001E089000AE089000A8
:108960007D0F07000017980011179800100F98004E
:10897000210F980087FC07000001EB00870D07001E
:10898000600F9800710F98000E1090009E109000DC
:10899000821F7800831F78006E099000FE09900006
:1089A0006B0E07004F01BE000002780081027800C4
:1089B0000000200001F02300040178008501780008
:1089C000A10E07000000E0000200340000002000BB
:1089D00001003700100020000000E0000A00320013
:1089E0007200470030027800A002780000002000EA
:1089F00001F023000401780085017800970E07003C
:108A0000100F9800210F98001E089000AE089000EB
:108A100060FC07006A024700144278000482FB00F1
:108A2000610242004223DD0084882F0006034200D9
:108A300036025000268258000C0039001E089000B3
:108A4000AE089000D2CC2C00C3DC2300AE0D070092
:108A5000100F9800210F98001400200076004700A6
:108A60001008420062450400000000001E0890004B
:108A7000AE08900047FC07006A02470014427800E5
:108A80000482FB004223DD0084882F00060342009D
:108A900036025000268258000A0031001E0890005D
:108AA000AE0890000200200003122400960D07007B
:108AB000100F9800210F9800140020007600470046
:108AC000100812006E0047001002780000202000FD
:108AD000000262004C0032006E0047001002780075
:108AE000008020000002620047003A006800470052
:108AF000100278006A00520002003400A00020003A
:108B00004007980078004700600F98001E0890000A
:108B1000AE0890001FFC07006E0A9000001A780053
:108B200001127800780247003400780024007000B9
:108B30001C00320078024700A2002000CF91DE0026
:108B400034007800A40078000002EB0047FC070026
:108B5000600250006082580012003A0014002000A9
:108B6000680047001008120078004700600F980066
:108B700030027800A0027800A200200004007800F3
:108B800085007800CF91DE000002EB0063FC070057
:108B90006E0A9000001A78000112780092450400D5
:108BA000000000006A004700104378000683FB00C5
:108BB000680247001400130013003D006A004700DC
:108BC000104278000482FB00680047001000520049
:108BD000801F78008EFA07002F00B1000001780096
:108BE000810178001E089000AE089000DA0E0700A0
:108BF000100F9800210F98006A0247006800470094
:108C000010407800004A78006800470010007800A3
:108C1000650240006C004700100812004E009000F2
:108C20000000E00007003A006E00470010027800E4
:108C3000008020000002620002003A002846040082
:108C400000000000140020006C0047001008120013
:108C50006E004700100078006302600003003200DD
:108C6000140020006C004700100812006E0047003E
:108C70001000780064026000390032006E00470086
:108C80001000780062026000140032006E0047009D
:108C9000100078006102600004003200D002200061
:108CA000004278005A46040000000000B002200094
:108CB000004278004EB89700044878001400200065
:108CC00068005700100842001400200070004700A0
:108CD0001008420088460400000000006E004700B3
:108CE0001000780061026000090032004EBA97005F
:108CF00000022000004A780014002000680057009D
:108D000010084200140020007000470010084200C4
:108D10006C00470010027800600052000E00340022
:108D20004EBA970000032000004A7800140020008B
:108D3000680057001008420014002000700047002F
:108D400010084200140020006C00470010081200B8
:108D500088460400000000002647040000000000D0
:108D60006E004700100078006802600012003A00B0
:108D70006C00470010027800600052000E003400C2
:108D80004EBA970000022000004A7800140020002C
:108D900068005700100842001400200070004700CF
:108DA00010084200140020006C0047001008120058
:108DB000B8460400000000006E0047001000780074
:108DC00062026000140032006E004700100078005C
:108DD0006102600004003200D002200000427800EE
:108DE000F846040000000000B002200000427800B5
:108DF0004EB897000448780014002000680057001F
:108E000010084200140020007000470010084200C3
:108E100026470400000000006E00470010007800A4
:108E200061026000090032004EBA97000002200083
:108E3000004A780014002000680057001008420023
:108E4000140020007000470010084200780047001E
:108E5000600F98001E089000AE0890004DFB0700C0
:108E60006E0A9000001A7800011278006E089000D7
:108E700030037800A00378006A00470010407800B3
:108E80000080FB004202DD0080882F0004024000C9
:108E900034017800A401780006007800870078008B
:108EA0000002EB009DFB0700060320004EBA97006E
:108EB000064A4000140020006800570010084200D5
:108EC0001400200070004700100842004E0090007F
:108ED0000000E00007003A006E0047001002780032
:108EE000008020000002620002003A0000480400F6
:108EF000000000004EBA9700E0022000004A78000F
:108F000014002000680057001008420014002000E0
:108F100070004700100842006A00470010427800C5
:108F20000482FB0068004700100812002E489000E1
:108F30000004E00021003200780047003003780090
:108F4000A00378006A024700144078006140500096
:108F5000004A78000080FB004202DD0080882F007C
:108F60000402400034017800A40178000600780073
:108F7000870078000002EB0068FB0700A4002000D7
:108F800004017800CF91DE000002EB0037FB070000
:108F9000060320004EBA9700004A43001400200048
:108FA00068005700100842001400200070004700BD
:108FB0001008420096470400000000004E00900098
:108FC0000000E0000E0032004EBA970000032000BF
:108FD000004A780014002000680057001008420082
:108FE0001400200070004700100842001400200008
:108FF0006800470010081200DE470400000000006F
:10900000040220006E004700100262000B003200D4
:109010004EBA970050042000004A78001400200047
:10902000680057001008420014002000700047003C
:109030001008420030480400000000004EBA9700BB
:1090400050062000004A78001400200068005700F5
:109050001008420014002000700047001008420071
:109060007600470010027800600052000E003D00BC
:109070007602470014007800600A10004EBA97008C
:10908000D0022000004A7800140020006800570039
:109090001008420014002000700047001008420031
:1090A00066480400000000004EBA9700B00220009D
:1090B000004A7800140020006800570010084200A1
:1090C000140020007000470010084200760047009E
:1090D0003017980010027800A2002000110009004B
:1090E0000202D800060320004EBA9700064A40004C
:1090F00068005700201798001000780061004000B9
:109100000017980040BF9F00140020007000470027
:10911000600F9800100842003E1090001002780086
:10912000A2002000110009000202D800010078000E
:10913000060320000E129000064A40000E10900018
:10914000140020002E10900010084200140020008F
:109150006E089000100842006E0047001000780072
:1091600068026000120032006C00470010027800B4
:10917000600052000E0034004EBA9700000220003A
:10918000004A7800140020006800570010084200D0
:109190001400200070004700100842006C004700D7
:1091A000100078006102500064079800F2FF3A0056
:1091B000F23E0400000000006E004700100278003C
:1091C0000020200000026200770032007600470095
:1091D000100278006000520005003D007600470054
:1091E000100078006102500068004700100812006B
:1091F00078004700600F98001E089000AE089000AD
:1092000064FA07006E0A9000001A780001127800D4
:109210006A02470010002000004A78006A004700F8
:10922000104278006A405200130032007804470070
:109230006A004700104078000080FB004202DD0019
:1092400080882F000403400038027800A8027800CC
:109250003600520026805A00020031003C490400CA
:1092600000000000140020006A004700104842007F
:109270000E490400000000006A0047001042780018
:109280000482FB00680047001000120020179800BD
:109290004007980078024700040078000017980003
:1092A00034007800A40078000001EB003B0B0700BD
:1092B000600F9800710F9800720247003400780028
:1092C000A4007800821F7800831F78006E09900048
:1092D000FE0990001E0C07004F01BE002E129000E8
:1092E000600F9800710F9800841F7800C8F807007D
:1092F0002F00B1006E0A9000FE0A90000401780071
:1093000085017800800B07000400200005F0230091
:109310000401780085017800500C07001DFA070051
:109320000E129000001A7800011278004E00900092
:109330000000E0001C00320078024700A20020007C
:10934000CF91DE0034007800A40078000002EB002A
:1093500046FA0700600250006082580012003A008E
:1093600078004700600F980030027800A002780073
:10937000A20020000400780085007800CF91DE0074
:109380000002EB0065FA07006E0A9000001A7800F0
:109390000112780014002000680047001008120035
:1093A00096490400000000006800470010027800A1
:1093B0006C0052000D003C0068004700100078006F
:1093C000801F780078F907002F00B1007203470072
:1093D00036027800A6027800040178008501780042
:1093E0001E0C0700100F9800210F98007202470012
:1093F00034007800A4007800020020000300200060
:10940000110C07000000E00002003A0000002000FC
:1094100001003700100020000000E0004000320092
:109420001E089000AE089000DAF9070060025000B4
:10943000608258003A003A00760047001002780037
:1094400061005200360034007600470010007800BA
:10945000801F78006EF807002F00B100000178002F
:10946000810178001E089000AE089000BA0C070039
:109470000002780081027800F0052700910824009E
:109480000401780085017800AC0B07000000E000C3
:1094900002003C0000002000010037001000200006
:1094A0000000E00005003200940020007600470034
:1094B00010081200644A040000000000840020002C
:1094C000760047001008120078004700600F9800EF
:1094D0007600470010007800801F78004CF80700E5
:1094E0002F00B10000017800810178001E08900073
:1094F000AE089000980C0700A6F907006E0A9000CD
:10950000001A7800011278000000200001002000FD
:10951000100F9800210F9800CA4A040000000000B4
:1095200078004700600F98001E089000AE08900079
:1095300098F907006E0A9000001A7800011278006E
:109540006E0890000002780034007800A4007800D3
:109550000001EB00910A0700600F9800710F98005E
:109560007202470034007800A4007800821F78005F
:10957000831F78006E099000FE099000740B0700AD
:109580004F01BE00100F9800210F9800000020002E
:10959000300F98006A02470010002000004A78004F
:1095A0006A004700104278006A40520013003200FF
:1095B000780447006A004700104078000080FB00F4
:1095C0004202DD0080882F0004034000380278004A
:1095D000A80278003600520026805A0002003100AE
:1095E000FE4A040000000000140020006A0047004A
:1095F00010484200D04A0400000000006A00470002
:10960000104278000482FB0068004700100242000C
:1096100076004700100242006C004700100812005C
:109620006E004700100278000080200000026200F7
:1096300005003A004E0090000000E00002003A00F1
:109640002A4B040000000000140020006C004700BA
:10965000100812006E0047001000780063026000DE
:1096600003003200140020006C00470010081200B4
:109670006E0047001000780064026000390032007C
:109680006E00470010007800620260001400320093
:109690006E00470010007800610260000400320094
:1096A000D0022000004278005C4B04000000000063
:1096B000B0022000004278004EB8970004487800BD
:1096C0001400200068005700100842001400200019
:1096D00070004700100842008A4B040000000000A0
:1096E0006E0047001000780061026000090032003F
:1096F0004EBA970000022000004A780014002000B3
:109700006800570010084200140020007000470055
:10971000100842006C004700100278006000520000
:109720000E0034004EBA970000032000004A780073
:1097300014002000680057001008420014002000A8
:109740007000470010084200140020006C00470021
:10975000100812008A4B040000000000284C04008E
:10976000000000006E0047001000780068026000F2
:1097700012003A006C0047001002780060005200AE
:109780000E0034004EBA970000022000004A780014
:109790001400200068005700100842001400200048
:1097A0007000470010084200140020006C004700C1
:1097B00010081200BA4B0400000000006E004700C1
:1097C0001000780062026000140032006E00470052
:1097D000100078006102600004003200D002200016
:1097E00000427800FA4B040000000000B0022000A4
:1097F000004278004EB8970004487800140020001A
:109800006800570010084200140020007000470054
:1098100010084200284C0400000000006E004700C1
:109820001000780061026000090032004EBA970013
:1098300000022000004A7800140020006800570051
:109840001008420014002000700047001008420079
:109850006A0347001642780010002000164B1000E3
:109860000404E0001F003200780047003003780055
:10987000A00378006A004700104078000080FB00D9
:109880004202DD0080882F0004024000340178008D
:10989000A401780006007800870078000002EB0041
:1098A0001EF90700A400200004017800CF91DE001B
:1098B0000002EB00EDF80700060320004EBA970007
:1098C000004A4300140020006800570010084200BE
:1098D000140020007000470010084200284C0400CB
:1098E000000000007600470010027800600052007F
:1098F0000E0034004EBA970000032000004A7800A2
:1099000014002000680057001008420014002000D6
:109910007000470010084200140020007600470045
:1099200010081200724C040000000000680047009C
:109930001002780068005200050034006A024700F7
:1099400080002000004A7800B04C040000000000B5
:109950006A0247006800470010407800004A78001B
:109960006A004700104278000482FB00680047004C
:10997000100812002E4890000004E00007003A0092
:109980006E00470010027800008020000002620094
:1099900002003A00E04C0400000000004EBA9700BC
:1099A000E0022000004A7800140020006800570000
:1099B0001008420014002000700047001008420008
:1099C00078004700600F98006A0047001040780058
:1099D0000080FB00801F78000DF707002F00B1000A
:1099E0001E099000AE099000C70907002F09070063
:1099F0006E0A9000001A7800011278002E4890003C
:109A00000004E000210032007800470030037800B5
:109A1000A00378006A0247001440780061405000BB
:109A2000004A78000080FB004202DD0080882F00A1
:109A30000402400034017800A40178000600780098
:109A4000870078000002EB00B4F80700A4002000B3
:109A500004017800CF91DE000002EB0083F80700DC
:109A6000060320004EBA9700004A4300140020006D
:109A700068005700100842001400200070004700E2
:109A800010084200FE4C0400000000004E00900050
:109A90000000E0000E0032004EBA970000032000E4
:109AA000004A7800140020006800570010084200A7
:109AB000140020007000470010084200140020002D
:109AC0006800470010081200464D04000000000026
:109AD0006E0047001000780068026000120032003B
:109AE0006C00470010027800600052000E00340045
:109AF0004EBA970000022000004A780014002000AF
:109B00006800570010084200140020007000470051
:109B1000100842006C0047001000780061025000FD
:109B200064079800F2FF3A00F23E040000000000D3
:109B3000040C20006E00470010026200600052001A
:109B40002A003A006E0047001000780070026000A2
:109B50000B00320078004700000478002EBB97000D
:109B60002EBA970040002000140A1000160078005A
:109B7000301C780020147800D64D0400000000004E
:109B800078004700000478002EBB97002EBA97009B
:109B900020002000140A1000160078001000780041
:109BA000CF80DE00001C78000114780078004700A8
:109BB00030027800A00278006000520060805A00F5
:109BC00008003D00340020006E00470010087200BD
:109BD0007802470034007800A4007800601A100072
:109BE000609218002A4E0400000000006E0047003A
:109BF00010007800700260000B003200780047000F
:109C0000000478002EBB97002EBA97004000200079
:109C1000140A100016007800301C78002014780018
:109C20002A4E04000000000078004700000478007D
:109C30002EBB97002EBA970020002000140A1000B7
:109C400016007800100078008000EB00001C7800FF
:109C5000011478006800470010027800600052008C
:109C600009003A007800470030027800A00278002E
:109C70006000520060805A0003003A001400200087
:109C80006800470010084200040C20006E004700E6
:109C90001000620080447800F84E040000000000CC
:109CA0006A02470010002000004A78006A0047005E
:109CB000104278006A4052001300320078044700D6
:109CC0006A004700104078000080FB004202DD007F
:109CD00080882F000403400038027800A802780032
:109CE0003600520026805A0002003100844E0400E3
:109CF00000000000140020006A00470010484200E5
:109D0000564E0400000000000E4F0400000000004A
:109D10006A02470010002000004A78006A004700ED
:109D20001042780068405200130032007804470067
:109D30006A004700104078000080FB004202DD000E
:109D4000008B2F000403400038027800A80278003E
:109D50003600520026805A0002003100BC4E04003A
:109D600000000000140020006A0047001048420074
:109D70008E4E0400000000000E4F040000000000A2
:109D80006A02470010002000004A78006A0047007D
:109D9000104278006C4052001300320078044700F3
:109DA0006A004700104078000080FB004202DD009E
:109DB000008D2F000403400038027800A8027800CC
:109DC0003600520026805A0002003100F44E040092
:109DD00000000000140020006A0047001048420004
:109DE000C64E0400000000000E4F040000000000FA
:109DF00060C05400AAFF3200040C200004C05400CC
:109E0000A7FF32000408200004C05400C0FF320045
:109E10000404200004C05400D9FF32006A00470047
:109E2000104378000683FB006802470014005300CB
:109E300006003D006A0247006800470010407800B5
:109E4000004A78003A4F0400000000006A00470012
:109E5000104378000683FB006802470014001300DB
:109E600004003D006A004700104078000080FB00BD
:109E7000400798006E0090000000E00007003200EC
:109E80006E0047001000780063026000030032009B
:109E9000140020006C004700100812006C004700FE
:109EA00010037800680247001400530006003400D5
:109EB00068004700100278006C004700100812008C
:109EC000684F0400000000000000200060079800B8
:109ED0006E00470010027800408C200000036200F2
:109EE000048420000400530008003A006E00900033
:109EF0000000E00003003200140020006C00470066
:109F000010081200AA4F0400000000006E00470075
:109F100010027800008C20000003620004882000FA
:109F2000040053000B003A006C0047001002780058
:109F30006200520005003400240020006C0047003D
:109F400010081200AA4F04000000000000002000CA
:109F5000600798006E0047001000780064026000FF
:109F60005C0032006E004700100078006202600062
:109F7000140032006E00470010007800610260009B
:109F800004003200D002200000427800CE4F0400CE
:109F900000000000B0022000004278004EB8970098
:109FA00004487800140020006800570010084200A0
:109FB00014002000700047001008420044500400C4
:109FC000000000006E004700100078006102600091
:109FD0000B0032004EBA970000022000004A7800C1
:109FE00014002000680057001008420014002000F0
:109FF00070004700100842004450040000000000B8
:10A000006E00470010027800008C20000003620000
:10A0100004882000040053001B003A004EBA970049
:10A0200000032000004A7800140020006800570058
:10A030001008420014002000700047001008420081
:10A04000040220006E00470010026200040032008B
:10A050008005200000427800345004000000000019
:10A0600080072000004278004EB89700044878002E
:10A07000140020006800570010084200140020005F
:10A0800070004700100842006E0090000000E000E1
:10A090000E0032004EBA970000032000004A7800FC
:10A0A000140020006800570010084200140020002F
:10A0B00070004700100842006C0047001000780054
:10A0C0006102500064079800F2FF3A004651040014
:10A0D000000000006E0090000000E000120032005E
:10A0E0006E00470010007800680260000E003A0021
:10A0F0004EBA970000022000004A780014002000A9
:10A10000680057001008420014002000700047004B
:10A11000100842006C0047001000780061025000F7
:10A1200064079800F2FF3A006E00470010007800C4
:10A1300062026000140032006E00470010007800D8
:10A140006102600004003200D0022000004278006A
:10A15000B050040000000000B0022000004278006F
:10A160004EB897000448780014002000680057009B
:10A170001008420014002000700047001008420040
:10A18000DE500400000000006E0047001000780060
:10A1900061026000090032004EBA97000002200000
:10A1A000004A7800140020006800570010084200A0
:10A1B0001400200070004700100842006E004700A5
:10A1C00010027800008C200000036200048420004C
:10A1D000040053000B003A004EBA97000003200021
:10A1E000004A780014002000680057001008420060
:10A1F000140020007000470010084200465104007F
:10A20000000000006E00470010027800008C200063
:10A210000003620004882000040053001B003A0081
:10A220004EBA970000032000004A78001400200076
:10A23000680057001008420014002000700047001A
:10A2400010084200040220006E0047001002620065
:10A2500004003200800520000042780036510400DE
:10A260000000000080072000004278004EB89700F0
:10A2700004487800140020006800570010084200CD
:10A280001400200070004700100842006A004700D8
:10A29000104378000683FB00680247001400130097
:10A2A0000B0034004EBA970000032000004A7800EB
:10A2B000140020006800570010084200140020001D
:10A2C00070004700100842004651040000000000E2
:10A2D0004E03900014002000680047001008120090
:10A2E0000600E0007E003200040C20006E004700F3
:10A2F00010006200405F98003C5204000000000023
:10A300007800470030037800A00378006800470019
:10A31000100078004202DD0080882F000402400017
:10A3200034017800A40178000600780087007800E6
:10A330000002EB0079F60700A40020000401780079
:10A34000CF91DE000002EB0048F607000603200074
:10A350006A024700064A40005A520400000000000A
:10A36000040220006E004700100262001700320055
:10A370007800470030037800A003780068004700A9
:10A38000100078004202DD00008B2F000402400024
:10A3900034017800A4017800060078008700780076
:10A3A0000002EB005DF607006F026000E0826000D3
:10A3B00000902F0004004000104278006A0047001F
:10A3C00004487800105204000000000078004700A4
:10A3D00030037800A0037800680047001000780080
:10A3E0004202DD00008B2F0004024000340178009F
:10A3F000A401780006007800870078000002EB00D6
:10A4000046F607006F026000E082600010912F00A6
:10A4100004004000104278006A00470004487800B9
:10A420005A52040000000000780047003003780012
:10A43000A003780068004700100078004202DD00A9
:10A44000008D2F000402400034017800A401780040
:10A4500006007800870078000002EB002FF6070066
:10A4600067036000040320006A00470004484300BB
:10A470005A520400000000004E5A90006040520002
:10A480009FFF3200060C20004E5A900006405200FA
:10A490009BFF3200060820004E5A900006405200F2
:10A4A000AFFF3200060420004E5A900006405200D2
:10A4B000DDFF32006A0247004EB89700144878006A
:10A4C000140020006800570010084200140020000B
:10A4D00070004700100842006851040000000000AE
:10A4E0006E00470010007800680260001200320021
:10A4F0006C00470010027800600052000E0034002B
:10A500004EBA970000022000004A78001400200094
:10A510006800570010084200140020007000470037
:10A52000100842006C0047001000780061025000E3
:10A5300064079800F2FF3A00F23E040000000000B9
:10A540000E0890000080FA00000006000400FA00E7
:10A55000E20047006A00570080087800811F7800F9
:10A56000901F780068005700901F780014F60700CD
:10A570006F00B100000F7800E80057009100400024
:10A5800000002000804878001E0078000080FA005B
:10A59000000006000200FA00680057001000780072
:10A5A000000F78001E0178001100200060004700B5
:10A5B000108840001204E00002003200D252040071
:10A5C000000000006000470090007800680057001D
:10A5D00010805000610050000080FA00000006006A
:10A5E0000200FA0068005700901F7800E9FF07009A
:10A5F0002F00B100000F780004060700600147003B
:10A600009200100008003600E0682000801F7800EB
:10A6100060002000801F7800170607004F00B1007F
:10A62000FC52040000000000680057009000780011
:10A63000314078000080FB00060032002022AF008D
:10A640001E5304000000000020118800185304006D
:10A65000000000000080FA00000006000000FA0080
:10A6600068005700901F780090922F00801F78009C
:10A6700020E62000801F7800B4FF07006F00B100C3
:10A6800020E62000801F7800D5FF07002F00B100D2
:10A690000080FA000000060050042000801F7800AF
:10A6A000EEFF07002F00B100000006000800FA00CE
:10A6B000D076800010079800E4DD2000CFA2DE00F5
:10A6C000E2D020003200120022801A000F003D006C
:10A6D000D2768000A0E5200010014100D2768800EB
:10A6E0006000510002003D0000002000D07688008C
:10A6F000D27680007B00510002003400B0012000BF
:10A70000D0768800E85E040000000000E4F6200037
:10A71000CFA2DE00E2D020003200120022801A0018
:10A720000F003400D2768000A0E520001001510017
:10A73000D27688006000510002003D000000200039
:10A74000D0768800D27680007B0051000200340071
:10A75000B0012000D0768800E85E04000000000010
:10A7600000002000000F7800E4F62000CFA2DE00F9
:10A7700062D020003200120022801A00040034004F
:10A7800010002000000F7800D853040000000000E3
:10A79000E4DD2000CFA2DE0062D0200032001200F3
:10A7A00022801A0002003D00F0FF2F00000F780009
:10A7B0006000470010017800E0E520001091B9002A
:10A7C000020F78006000510081053200D2768000CF
:10A7D0007B0051000600320010002000B077880096
:10A7E000B0012000801F780023F007002F00B10087
:10A7F000365E0400000000007276800083768000E0
:10A800000000200001F823000F0707000000E0000F
:10A81000020034000000200001003700100020007A
:10A820000000E000060032006000470010017800E0
:10A830006000510002003D00485404000000000088
:10A84000727680008376800000C02300C1612400FE
:10A85000BA0607000000E00002003C0000002000F3
:10A8600001003700100020000000E0000600320068
:10A8700060004700100178006000510002003400C1
:10A8800048540400000000005A5404000000000076
:10A890001E007800CF80DE000081EB00BF050700BE
:10A8A0007276800083768000EC0607007076880060
:10A8B00081768800E25E040000000000427580009E
:10A8C00053758000A0702D0031C22300DE06070002
:10A8D0000000E0000200340000002000010037000A
:10A8E000100020000000E000060032006000470079
:10A8F000100178006000510002003D00AA540400DD
:10A9000000000000427580005375800000002000A8
:10A9100001F82300890607000000E00002003C0067
:10A920000000200001003700100020000000E000BF
:10A9300006003200600047001001780060005100FE
:10A9400002003400AA54040000000000C2540400B5
:10A95000000000001E007800CF80DE000081EB00C8
:10A960008E050700A2702D0033C22300E605070004
:10A970004275800053758000B80607004075880056
:10A9800051758800E25E0400000000004270800003
:10A9900053708000D0CC2C00C1E42300AA0607002D
:10A9A0000000E00002003400000020000100370039
:10A9B000100020000000E0000600320060004700A8
:10A9C000100178006000510002003D0012550400A3
:10A9D000000000004270800053708000303323007C
:10A9E000F1192400550607000000E00002003C00B9
:10A9F0000000200001003700100020000000E000EF
:10AA0000060032006000470010017800600051002D
:10AA10000200340012550400000000002A55040012
:10AA2000000000001E007800CF80DE000081EB00F7
:10AA30005A050700D2CC2C00C3DC2300B205070066
:10AA400042708000537080008406070040708800C8
:10AA500051708800E25E0400000000003270800047
:10AA600061005100060034006000470010017800CA
:10AA70006000510002003D00585504000000000035
:10AA80005409200062E020001200120006003D0080
:10AA9000600047001001780060005100020034009F
:10AAA000585504000000000060550400000000003C
:10AAB000600047001001780060E0200010084100AD
:10AAC000E25E0400000000005276800063768000A1
:10AAD0000000200001F823005B0607000000E000F2
:10AAE00002003500000020000100370010002000A7
:10AAF0000000E0000600320060004700100178000E
:10AB00006000510002003D00B0550400000000004C
:10AB1000527680006376800000C02300C16124006B
:10AB2000060607000000E00002003C0000002000D4
:10AB300001003700100020000000E0000600320095
:10AB400060004700100178006000510002003400EE
:10AB5000B055040000000000C255040000000000D1
:10AB60001E007800CF80DE000081EB000B0507009F
:10AB700052768000637680003806070050768800A1
:10AB800061768800E25E040000000000027280002E
:10AB900013728000D0CC2C00C1DC23002A060700F1
:10ABA0000000E00002003500000020000100370036
:10ABB000100020000000E0000600320060004700A6
:10ABC000100178006000510002003D0012560400A0
:10ABD000000000000272800013728000D0CC2C00B4
:10ABE000712C2400D50507000000E00002003C00A5
:10ABF0000000200001003700100020000000E000ED
:10AC0000060032006000470010017800600051002B
:10AC10000200340012560400000000002A5604000E
:10AC2000000000001E007800CF80DE000081EB00F5
:10AC3000DA040700D2CC2C00C3DC23003205070065
:10AC40000272800013728000040607000072880000
:10AC500011728800E25E040000000000E0768000CF
:10AC6000F17680000200200003002000B3050700F9
:10AC70000000E00002003C0000002000010037005E
:10AC8000100020000000E0000600320060004700D5
:10AC9000100178006000510002003D007A56040067
:10ACA00000000000E2768000F376800000002000C3
:10ACB00041242400A10507000000E00002003C0040
:10ACC0000000200001003700100020000000E0001C
:10ACD000060032006000470010017800600051005B
:10ACE000020034007A560400000000008C56040074
:10ACF000000000001E007800CF80DE000081EB0025
:10AD0000A6040700E2768000F3768000D3050700F2
:10AD1000E0768800F1768800E25E04000000000022
:10AD2000E2718000F3718000D0CC2C00C1DC2300E4
:10AD3000C50507000000E00002003500000020000B
:10AD400001003700100020000000E0000600320083
:10AD500060004700100178006000510002003D00D3
:10AD6000DC56040000000000E2718000F3718000F6
:10AD7000D0CC2C00712C2400700507000000E000EE
:10AD800002003C00000020000100370010002000FD
:10AD90000000E0000600320060004700100178006B
:10ADA0006000510002003400DC5604000000000086
:10ADB000F4560400000000001E007800CF80DE0082
:10ADC0000081EB0075040700D2CC2C00C3DC23000B
:10ADD000CD040700E2718000F37180009F05070039
:10ADE000E0718800F1718800E25E0400000000005C
:10ADF0000277800013778000D0CC2C00C1DC2300C8
:10AE0000910507000000E00002003500000020006E
:10AE100001003700100020000000E00006003200B2
:10AE200060004700100178006000510002003D0002
:10AE30004457040000000000027780001377800070
:10AE4000D0CC2C00712C24003C0507000000E00051
:10AE500002003C000000200001003700100020002C
:10AE60000000E0000600320060004700100178009A
:10AE7000600051000200340044570400000000004C
:10AE80005C570400000000001E007800CF80DE0048
:10AE90000081EB0041040700D2CC2C00C3DC23006E
:10AEA0009904070002778000137780006B05070084
:10AEB0000077880011778800E25E0400000000003F
:10AEC00020778000317780000200200003002000FE
:10AED0001A0507000000E00002003C00000020000E
:10AEE00001003700100020000000E00006003200E2
:10AEF00060004700100178006000510002003D0032
:10AF0000AC570400000000002277800033778000F7
:10AF10000000200041242400080507000000E00094
:10AF200002003C000000200001003700100020005B
:10AF30000000E000060032006000470010017800C9
:10AF40006000510002003400AC5704000000000013
:10AF5000BE570400000000001E007800CF80DE0015
:10AF60000081EB000D04070022778000337780001A
:10AF70003A0507002077880031778800E25E0400F8
:10AF80000000000042728000537280000000200028
:10AF900001F823002C0507000000E0000200350046
:10AFA0000000200001003700100020000000E00039
:10AFB0000600320060004700100178006000510078
:10AFC00002003D000E5804000000000042728000A4
:10AFD0005372800000002000612C2400D704070079
:10AFE0000000E00002003C000000200001003700EB
:10AFF000100020000000E000060032006000470062
:10B000001001780060005100020034000E58040066
:10B010000000000020580400000000001E0078001E
:10B02000CF80DE000081EB00DC030700427280006D
:10B030005372800009050700407288005172880031
:10B04000E25E040000000000227280003372800083
:10B05000D0CC2C00C1DC2300FB0407000000E00082
:10B060000200350000002000010037001000200021
:10B070000000E00006003200600047001001780088
:10B080006000510002003D00705804000000000004
:10B090002272800033728000D0CC2C00712C2400EE
:10B0A000A60407000000E00002003C0000002000B1
:10B0B00001003700100020000000E0000600320010
:10B0C0006000470010017800600051000200340069
:10B0D00070580400000000008858040000000000C0
:10B0E0001E007800CF80DE000081EB00AB0307007C
:10B0F000D2CC2C00C3DC23000304070022728000A2
:10B1000033728000D50407002072880031728800F5
:10B11000E25E040000000000A2718000B3718000B4
:10B120000000200001F82300C70407000000E00031
:10B130000200350000002000010037001000200050
:10B140000000E000060032006000470010017800B7
:10B150006000510002003D00D858040000000000CB
:10B16000A2718000B371800000002C009147240080
:10B17000720407000000E00002003C000000200014
:10B1800001003700100020000000E000060032003F
:10B190006000470010017800600051000200340098
:10B1A000D858040000000000EA5804000000000025
:10B1B0001E007800CF80DE000081EB0077030700DF
:10B1C000A2718000B3718000A4040700A071880000
:10B1D000B1718800E25E040000000000C2718000CE
:10B1E000D37180000000200001F8230096040700BE
:10B1F0000000E000020035000000200001003700E0
:10B20000100020000000E00006003200600047004F
:10B21000100178006000510002003D003A5904001E
:10B2200000000000C2718000D37180000000200087
:10B23000612C2400410407000000E00002003C00F3
:10B240000000200001003700100020000000E00096
:10B2500006003200600047001001780060005100D5
:10B26000020034003A590400000000004C59040068
:10B27000000000001E007800CF80DE000081EB009F
:10B2800046030700C2718000D37180007304070079
:10B29000C0718800D1718800E25E040000000000E7
:10B2A00042778000537780000000200001F82300DF
:10B2B000650407000000E0000200350000002000E7
:10B2C00001003700100020000000E00006003200FE
:10B2D00060004700100178006000510002003D004E
:10B2E0009C590400000000004277800053778000E2
:10B2F0000000200031332400100407000000E000AB
:10B3000002003C0000002000010037001000200077
:10B310000000E000060032006000470010017800E5
:10B3200060005100020034009C590400000000003D
:10B33000AE590400000000001E007800CF80DE003F
:10B340000081EB00150307004277800053778000EF
:10B35000420407004077880051778800E25E0400CD
:10B36000000000003276800043768000000020005C
:10B3700001122400340407000000E0000200350040
:10B380000000200001003700100020000000E00055
:10B390000600320060004700100178006000510094
:10B3A00002003D00FE5904000000000032768000DB
:10B3B0004376800000C02300C1612400DF03070042
:10B3C0000000E00002003C00000020000100370007
:10B3D000100020000000E00006003200600047007E
:10B3E000100178006000510002003400FE59040092
:10B3F00000000000145A040000000000A200200019
:10B40000600047001090B900CF80DE000081EB00A3
:10B41000E202070032768000437680000F040700C6
:10B420003076880041768800E25E0400000000006B
:10B43000D2728000600051000600340060004700B6
:10B44000100178006000510002003D00405A0400E5
:10B4500000000000D27280006000510006003D0034
:10B4600060004700100178006000510002003400C5
:10B47000405A040000000000465A0400000000008A
:10B480006000470010007800D0728800E25E04007F
:10B4900000000000F27280006000510006003400DD
:10B4A00060004700100178006000510002003D007C
:10B4B000725A040000000000F27280006000510027
:10B4C00006003D0060004700100178006000510058
:10B4D00002003400725A040000000000785A040090
:10B4E000000000006000470010007800F072880043
:10B4F000E25E040000000000127580006000510050
:10B500000600340060004700100178006000510020
:10B5100002003D00A45A04000000000012758000E3
:10B520006000510006003C006000470010017800F8
:10B530006000510002003400A45A04000000000022
:10B54000AC5A0400000000006000470010017800C1
:10B5500020EA200010084100E25E04000000000024
:10B56000026980006000510006003400600047005E
:10B57000100178006000510002003D00DA5A04001A
:10B580000000000004698000823E2000020052009A
:10B5900006003D0060004700100178006000510087
:10B5A00002003400DA5A040000000000E25A0400ED
:10B5B00000000000600047001001780000D2200069
:10B5C00010084100E25E040000000000926E80005E
:10B5D0006000510006003400600047001001780050
:10B5E0006000510002003D000E5B040000000000FE
:10B5F000926E80006000510006003C006000470031
:10B600001001780060005100020034000E5B04005D
:10B61000000000001A5B040000000000600047000A
:10B620001001780020DD2000100841005DEC0700CB
:10B63000B9EE0700E25E04000000000062778000BF
:10B6400065005100060034006000470010017800DA
:10B650006000510002003D00485B04000000000053
:10B66000C4032000C2EE20001200120006003D00BC
:10B6700060004700100178006000510002003400B3
:10B68000485B040000000000505B04000000000064
:10B690006000470010017800C0EE20001008410053
:10B6A000E25E040000000000600047001001780026
:10B6B0006000510006003400000020002070880067
:10B6C00010002000801F78001CEF07002F00B10041
:10B6D000E25E040000000000727780008377800043
:10B6E000C05A2C0071722300570307000000E000CD
:10B6F000020035000000200001003700100020008B
:10B700000000E000060032006000470010017800F1
:10B710006000510002003D00B85B04000000000022
:10B720007277800083778000D0CC2C00C1DC2300AE
:10B73000020307000000E00002003C0000002000BF
:10B7400001003700100020000000E0000600320079
:10B7500060004700100178006000510002003400D2
:10B76000B85B040000000000D05B04000000000093
:10B770001E007800CF80DE000081EB00070207008A
:10B78000C25A2C00737223005F0207007277800098
:10B790008377800031030700707788008177880005
:10B7A000E25E04000000000092778000A377800032
:10B7B000F026210031A82300230307000000E00049
:10B7C00002003500000020000100370010002000BA
:10B7D0000000E00006003200600047001001780021
:10B7E0006000510002003D00205C040000000000E9
:10B7F00092778000A37780000000200001F82300EA
:10B80000CE0207000000E00002003C000000200023
:10B8100001003700100020000000E00006003200A8
:10B820006000470010017800600051000200340001
:10B83000205C040000000000385C040000000000F0
:10B840001E007800CF80DE000081EB00D3010700EE
:10B85000F226210033A823002B02070092778000F4
:10B86000A3778000FD02070090778800A177880009
:10B87000E25E040000000000F274800060005100ED
:10B88000060034006000470010017800600051009D
:10B8900002003D00665C04000000000084022000FD
:10B8A000E2E920001200120006003D00600047009F
:10B8B000100178006000510002003400665C040052
:10B8C00000000000705C040000000000F2748000C2
:10B8D0006000470010004100F07488000075880087
:10B8E000E25E0400000000006000470010007800E5
:10B8F000610050000200320000002000010037000B
:10B900001000200060758800E25E04000000000066
:10B91000600047001001780060005100CF00340043
:10B9200000C02F00F1072000200798003107980081
:10B9300020002000801F7800E0EC2000801F7800AD
:10B9400064004700801F7800E8EE07006F00B10038
:10B9500020002000801F780080EA2000801F7800EF
:10B9600064004700801F7800E0EE07006F00B10020
:10B9700020002000801F780080E02000801F7800D9
:10B9800064004700801F7800D8EE07006F00B10008
:10B9900010002000801F780060E02000801F7800E9
:10B9A00064004700801F7800D0EE07006F00B100F0
:10B9B00020002000801F7800A0EC2000801F78006D
:10B9C00064004700801F7800C8EE07006F00B100D8
:10B9D00020002000801F780000E42000801F7800F5
:10B9E00064004700801F7800C0EE07006F00B100C0
:10B9F00020002000801F7800C0ED2000801F78000C
:10BA000064004700801F7800B8EE07006F00B100A7
:10BA100020002000801F7800C0E32000801F7800F5
:10BA200064004700801F7800B0EE07006F00B1008F
:10BA300020002000801F780000EE2000801F78008A
:10BA400064004700801F7800A8EE07006F00B10077
:10BA500020002000801F780040EE2000801F78002A
:10BA600064004700801F7800A0EE07006F00B1005F
:10BA700020002000801F780080E42000801F7800D4
:10BA800064004700801F780098EE07006F00B10047
:10BA900020002000801F780040E42000801F7800F4
:10BAA00064004700801F780090EE07006F00B1002F
:10BAB00020002000801F780040E32000801F7800D5
:10BAC00064004700801F780088EE07006F00B10017
:10BAD00020002000801F780080EE2000801F78006A
:10BAE00064004700801F780080EE07006F00B100FF
:10BAF00020002000801F780080E32000801F780055
:10BB000064004700801F780078EE07006F00B100E6
:10BB100020002000801F780060EC2000801F78004B
:10BB200064004700801F780070EE07006F00B100CE
:10BB300010002000801F7800A0E52000801F780002
:10BB400064004700801F780068EE07006F00B100B6
:10BB500010002000801F7800E0E52000801F7800A2
:10BB600064004700801F780060EE07006F00B1009E
:10BB700010002000801F780020EA2000801F78003D
:10BB800064004700801F780058EE07006F00B10086
:10BB900010002000801F780000D22000801F780055
:10BBA00064004700801F780050EE07006F00B1006E
:10BBB00010002000801F780020DD2000801F78000A
:10BBC00064004700801F780048EE07006F00B10056
:10BBD00010002000801F7800C0EE2000801F780039
:10BBE00064004700801F780040EE07006F00B1003E
:10BBF00020002000801F7800E0EE2000801F7800E9
:10BC000064004700801F780038EE07006F00B10025
:10BC100020002000801F780020EF2000801F780087
:10BC200064004700801F780030EE07006F00B1000D
:10BC300020002000801F7800E0E92000801F7800AD
:10BC400064004700801F780028EE07006F00B100F5
:10BC500000002000B07788002FED0700E25E0400AE
:10BC600000000000E25E040000000000D2768000C8
:10BC700060005100E0FA3200D2768000610051008D
:10BC80000EFB3200D2768000620051003FFB320092
:10BC9000D27680006300510070FB3200D2768000C3
:10BCA0006400510088FB3200D276800065005100AC
:10BCB000B6FB3200D276800066005100E7FB32000E
:10BCC000D27680006700510015FC3200D2768000E9
:10BCD0006800510046FC3200D276800069005100B5
:10BCE00077FC3200D27680006A005100A5FC320059
:10BCF000D27680006B005100D3FC3200D2768000F7
:10BD00006C00510004FD3200D27680006D005100BD
:10BD100032FD3200D27680006E00510060FD3200AC
:10BD2000D27680006F0051008EFD3200D276800006
:10BD300070005100BEFD3200D276800071005100CB
:10BD4000D4FD3200D276800072005100EAFD32004C
:10BD5000D27680007300510001FE3200D27680005E
:10BD60007400510019FE3200D27680007500510037
:10BD700032FE3200D2768000760051004AFE320058
:10BD8000D27680007700510053FE3200D2768000D8
:10BD90007800510084FE3200D27680007900510094
:10BDA000B5FE3200D27680007A005100CEFE32001D
:10BDB000D27680007B005100D5FE3200325E040056
:10BDC00000000000DA0EF800ABEA07002F00B10017
:10BDD0006200470010027800A2ED2000120052001D
:10BDE0000700320062004700901F7800A2EA0700B7
:10BDF0002F00B100DA0EF8009FEA07002F00B10013
:10BE000025FA07000080FA000000060020C2A90001
:10BE10002022AF00085F040000000000F00F2000A7
:10BE2000201188002002AE00125F04000000000014
:10BE300020118000F10F20000104E100F3FF3A001F
:10BE400020C2A9002022AF00225F040000000000F1
:10BE50000000EB00201188002002AE002C5F0400DF
:10BE60000000000020118000F000B200110020004E
:10BE70000008DD00000006000000FA004EB8970040
:10BE8000BEB897000000E00004003200FA3F09004D
:10BE9000000000000000E900FAFF370001800900FF
:10BEA000000000000080FA00000006000000FA0018
:10BEB00002000700CA5F0400000000000001BE008D
:10BEC0001F0007000470A70003F0A1006509B1007E
:10BED000160032000D0035006828E100060035002C
:10BEE000F0FF2F00F1FF27000300E00013003B00EC
:10BEF000010028000000050000004000818048008B
:10BF00008502E900FCFF3A0008003700F88F420084
:10BF100002003C008000EB00000005008100D10021
:10BF20000080D3008502E800FCFF3A000300E00037
:10BF300002003B0060001000E080180000000600D6
:10BF4000C70ADE00F107B200F50FB20008003200A8
:10BF5000E1CF4200020032000170A0002400050081
:10BF6000810F700001003200040805004400050044
:10BF7000810F700002003A00140005008502E900FC
:10BF80000000400081C04800FCFF3B000170A000A1
:10BF9000240005000080FA00000006000000FA00FE
:10BFA0000200070080600400000000000200E000C2
:10BFB00006003A000005EB000100E0000F003E0023
:10BFC0000000E000270032000C0037000105780077
:10BFD0000100E0000400350008003C000000E00023
:10BFE000200032000500370060001000E0801800DB
:10BFF00002003B0001F02C001A0037000004BE00D4
:10C000006011B8006B0920000982CF0002003900DE
:10C010000882CF000441B000694252000E00320095
:10C0200008003B0082817100610164008904D10035
:10C030000884D3008B05E8000442E800F9FF3A00C9
:10C04000050037000804440089844C008B05E90092
:10C050000442E900FBFF3A00030007000AF0A700D2
:10C0600001F0A00000000600810020006180550062
:10C070000B003D000B00200061FE2F000100E100DD
:10C080001D00340082817100610164008904D100C7
:10C090000884D3000000E800FAFF3A007100200095
:10C0A00061006400030070000200600009003200BB
:10C0B00061044400E0844C000988A50005003200BA
:10C0C0008B05E8006808E10002003A008904D1000D
:10C0D0000884D300F20F20000258E10005003D0063
:10C0E000C75DDD00F907B20089807500080078009F
:10C0F000000006000BF827008B0078000000050008
:10C100000080FA00000006000000FA0002000700AC
:10C110009A61040000000000889FBE008A9FBE0054
:10C120008C1F7800300007003700330003866C0056
:10C130006450E100240032006420E1002700320056
:10C140006150E100220032006120E1002100320054
:10C150008B854200EB07B1000134B800003AB8000B
:10C160000804420089844A00013AB8000030B8004F
:10C170008880400009014A000400330000004000AC
:10C1800081804800020149008B05E900C909DD00F2
:10C19000830170000100320013002000C814DE008B
:10C1A0004814DD004709DE001200B200C808DE00B6
:10C1B000088470002400070001F0A1000CF0A70023
:10C1C00001F0A000190037006120E1001B003200DF
:10C1D0000801BE000200BE00F7FF37006150E10019
:10C1E000FCFF3A00150037000004BE003C000700C9
:10C1F0000003BE000405BE000200BE0038000700B8
:10C20000844F7500000006000200BE006450E1008B
:10C21000050036006420E100020036000968A30032
:10C2200001003A000800BE000160A0004F0678003F
:10C230004F05BE004F04BE0000000600F0FF2F00B7
:10C24000F1FF2700F9FF37008100200061805500D1
:10C250000B003D000B00200061FE2F000100E100FB
:10C260001D00340082817100610164008904D100E5
:10C270000884D3000000E800FAFF3A0071002000B3
:10C2800061006400030070000200600009003200D9
:10C2900061044400E0844C000988A50005003200D8
:10C2A0008B05E8006808E10002003A008904D1002B
:10C2B0000884D300F20F20000258E10005003D0081
:10C2C000C75DDD00F907B2008980750008007800BD
:10C2D000000006000BF827008B0078000000050026
:10C2E000C70ADE00F107B200F50FB2000800320005
:10C2F000E1CF4200020032000170A00024000500DE
:10C30000810F7000010032000408050044000500A0
:10C31000810F700002003A00140005008502E90058
:10C320000000400081C04800FCFF3B000170A000FD
:10C33000240005000080FA00000006000000FA005A
:10C34000F4FF2F00070007000080FA00000006003D
:10C350000000FA0003F0A200400007000080FA008D
:10C36000000006000000FA0002000700206204003E
:10C3700000000000841F7800140007004F007800C0
:10C3800011003300F0FF2F00838F6C0006003B008C
:10C39000040565000A00A7000800370009F0A600A0
:10C3A0001000200008003700820F5400838F5C00CB
:10C3B000030039001000200001003E0000002000B2
:10C3C00009F0A7000000EA00000006000004BE001B
:10C3D000060007000003BE000405BE000200BE0008
:10C3E00002000700844F750000000600C70ADE0047
:10C3F000F107B200F50FB20008003200E1CF4200B1
:10C40000020032000170A00024000500810F7000BE
:10C41000010032000408050044000500810F70008F
:10C4200002003A00140005008502E9000000400007
:10C4300081C04800FCFF3B000170A0002400050003
:10C440000080FA00000006000000FA00140020003E
:10C45000C4FF07000080FA00000006000000FA0098
:10C46000020007009663040000000000889FBE00E1
:10C470008A9FBE008C1F78005900070060003300BF
:10C480006450E1004F0032006420E10052003200AD
:10C4900003826C0007003B000905D0000306D000B2
:10C4A000820F54000C065D000200390002003200C9
:10C4B00089017800030678008582550004003D005C
:10C4C0000003FD008103FD008502EA008B85420028
:10C4D000840F720002003B0060001000E080180032
:10C4E0006011B8000005EB007A28E1000A0039006D
:10C4F00006007800C75DDD00F707B2008780750091
:10C500002D003700828171000A017800610560000A
:10C510008180D1000080D3008502E900F9FF3B0053
:10C52000060440008784480002003B0060041400B9
:10C53000E0841C000988A300070032008A81710092
:10C5400082817100610164008904D1000884D300F4
:10C550008B05E800170037000978A30013003A00A4
:10C560000B00E000130034008B05E90008044400D0
:10C5700089844C000A4474000978A3000D003A0035
:10C580000B00E000070034008B05E90008044400BC
:10C5900089844C0001003A000B0020000978A300B8
:10C5A000F7FF32000001EB000200370082817100CA
:10C5B0000A017800220007000CF0A70001F0A0009B
:10C5C000180037006420E10002003A00838F6C00FD
:10C5D000180033000801BE000200BE001100370041
:10C5E0000004BE003C0007000003BE000405BE00BE
:10C5F0000200BE0038000700844F750000000600EE
:10C600000200BE006450E100050036006420E10035
:10C61000020036000968A30001003A000800BE00CD
:10C620000160A0004F0678004F05BE004F04BE0019
:10C6300000000600F0FF2F00F1FF2700F9FF370090
:10C6400081002000618055000B003D000B002000A0
:10C6500061FE2F000100E1001D00340082817100A5
:10C66000610164008904D1000884D3000000E8005F
:10C67000FAFF3A00710020006100640003007000BE
:10C68000020060000900320061044400E0844C00B4
:10C690000988A500050032008B05E8006808E10064
:10C6A00002003A008904D1000884D300F20F200070
:10C6B0000258E10005003D00C75DDD00F907B2004A
:10C6C0008980750008007800000006000BF827003C
:10C6D0008B00780000000500C70ADE00F107B200F9
:10C6E000F50FB20008003200E1CF42000200320034
:10C6F0000170A00024000500810F700001003200CD
:10C700000408050044000500810F700002003A0093
:10C71000140005008502E9000000400081C04800C7
:10C72000FCFF3B000170A000240005000080FA001F
:10C73000000006000000FA00020AB800800278003B
:10C740000200B80081004200032AB80081004200C4
:10C750000080FA00000006000000FA000200070056
:10C76000DE64040000000000889FBE008A9FBE00B7
:10C770008C1F78003E0007004500330003866C00E4
:10C780006450E1002E0032006420E10033003200EA
:10C790006150E1002F0032006120E10031003200E1
:10C7A00085855500EB07B000090020000804200033
:10C7B000050037000804440089844C000A00310059
:10C7C0000603430087834B000001530081815B0017
:10C7D000F8FF33000203BE000800A0000804440074
:10C7E00089844C00F6FF3900C639DD0083017300EF
:10C7F00001003200130020008904D1000884D30016
:10C800000998A300050032000800A7000300A0005B
:10C810008904D1000884D3008B05E8008904D10085
:10C820000884D3000001EB000281D2002800070039
:10C8300001F0A1000CF0A70001F0A0001D003700DE
:10C840006420E1001F0032000801BE000200BE00AB
:10C85000F7FF37006120E1001A0032006000B800E5
:10C86000F3FF37000000200001F82700F0FF370039
:10C870000004BE003C0007000003BE000405BE002B
:10C880000200BE0038000700844F7500000006005B
:10C890000200BE006450E100050036006420E100A3
:10C8A000020036000968A30001003A000800BE003B
:10C8B0000160A0004F0678004F05BE004F04BE0087
:10C8C00000000600F0FF2F00F1FF2700F9FF3700FE
:10C8D00081002000618055000B003D000B0020000E
:10C8E00061FE2F000100E1001D0034008281710013
:10C8F000610164008904D1000884D3000000E800CD
:10C90000FAFF3A007100200061006400030070002B
:10C91000020060000900320061044400E0844C0021
:10C920000988A500050032008B05E8006808E100D1
:10C9300002003A008904D1000884D300F20F2000DD
:10C940000258E10005003D00C75DDD00F907B200B7
:10C950008980750008007800000006000BF82700A9
:10C960008B00780000000500C70ADE00F107B20066
:10C97000F50FB20008003200E1CF420002003200A1
:10C980000170A00024000500810F7000010032003A
:10C990000408050044000500810F700002003A0001
:10C9A000140005008502E9000000400081C0480035
:10C9B000FCFF3B000170A000240005000080FA008D
:10C9C000000006000F802000E0BF2000000188006A
:10C9D0004440A80000002000A0018800AA00FA003E
:10C9E00060004700B1942F0004000900315878001E
:10C9F0006500470001952F000E00090031587800AE
:10CA000074004700F1952F00390009003158780073
:10CA1000E00420000000470091992F001800090051
:10CA2000315878007006200000004700219B2F003D
:10CA30000300090031587800B006200000004700CC
:10CA4000619B2F0005000900315878001007200075
:10CA500000004700C19B2F000700090031587800F3
:10CA600000002000503F9800000020000087980040
:10CA700000772000400E880000002000C0168800CB
:10CA8000E4FF2F00A02D200010086200E0E020004D
:10CA9000801F780010002000801F7800F6FC07003F
:10CAA0004F00B10014002000A02D200010087200DB
:10CAB000002C210001002000801F7800811F7800D9
:10CAC00015CF07004F00B10004402000C020200017
:10CAD000100872000000200000979800000A200053
:10CAE0000000470010027800620052000F003D0075
:10CAF000C409200004024700000A2000000047008B
:10CB0000100078004100DD0000024200000020001B
:10CB1000000A780014002000000A200000004700EE
:10CB2000100842006E6504000000000000002000B4
:10CB300060758800000020000097980050CF070023
:10CB400064CF070000002000CF80DE00207888003E
:10CB50003178880000002000010020000078880063
:10CB6000117888000000200001002000E077880094
:10CB7000F17788000000200001002000C0778800C5
:10CB8000D177880060EA2000CF80DE00B06888009E
:10CB9000C168880060EA20000100200090688800D9
:10CBA000A168880060EA2000010020003068880049
:10CBB0004168880060EA2000010020007068880059
:10CBC0008168880010002000107588000000200097
:10CBD00001002000107688002176880000002000E7
:10CBE00001002000D06A8800E16A8800000020006F
:10CBF000010020007072880081728800000020000F
:10CC000001002000A0728800B1728800000020009E
:10CC10000100200020758800317588000000200088
:10CC200001002000F06A8800016B880000002000ED
:10CC300001002000A0708800B17088000000200072
:10CC400001002000806A8800916A880000002000AE
:10CC500001002000606A8800716A880000002000DE
:10CC600001002000106A8800216A8800000020006E
:10CC700001002000406A8800516A880000002000FE
:10CC80000100200060879800718798000000200054
:10CC90000100200040879800518798000000200084
:10CCA0000100200080708800917088000000200042
:10CCB00001002000C0708800D170880000002000B2
:10CCC0000100200060708800717088000000200062
:10CCD00001002000106F8800216F880000002000F4
:10CCE00001002000D06E8800E16E88000000200066
:10CCF00001002000F06E8800016F8800600047008E
:10CD0000801F780060DE2000801F78006CCF070055
:10CD10004F00B100000020000071880000002000DA
:10CD2000F070880000002000E07088000000200003
:10CD300010708800000020000070880000002000B3
:10CD4000F06F880000002000E069880000002000EB
:10CD5000F069880000002000006A880000002000C0
:10CD60000100200090768800A17688000000200055
:10CD7000010020004DFC0700907188008071880040
:10CD80009072880060728800CF80DE000081EB0026
:10CD900082FC0700707588008175880030718800FA
:10CDA000417188005071880061718800107188009D
:10CDB0002171880064D4200000022000004A78001D
:10CDC00074D4200000022000004A780074D22000B1
:10CDD00000022000004A780060EA2000CF80DE00D8
:10CDE000B0688800C168880060EA20000100200067
:10CDF00090688800A168880060EA20000100200097
:10CE0000306888004168880060EA20000100200046
:10CE1000706888008168880000002000CF80DE00F4
:10CE2000106988002169880000002000F0688800EF
:10CE300000002000E068880000002000D068880022
:10CE400000002000B07788000000200030879800A4
:10CE500000002000208798000000200070718800EA
:10CE600000002000C06A88000000200020708800B8
:10CE700000002000106B880000002000C0768800B1
:10CE800000002000B076880000002000703F98006D
:10CE900000002000D0768800000020005068880044
:10CEA0000000200010879800A0C52F00F107200087
:10CEB000208F9800318F980000002000CF80DE0086
:10CEC000408F9800518F980010002000806E8800DD
:10CED000100020006068880064D22000400020001C
:10CEE000004A780000002000006888000000200050
:10CEF00010688800000020002068880000102000D2
:10CF0000801F780000002000801F780000002000B3
:10CF1000801F780000082000801F7800000020009B
:10CF2000801F780020002000801F78000000200073
:10CF3000801F780000022000801F780016CF0700B5
:10CF40000F01B100F4FF2D00202220001008620024
:10CF500004002400202220001008720000C02F00CE
:10CF6000F1072000008F9800118F9800200020000A
:10CF7000801F7800E0EC2000801F7800000920006E
:10CF800000004700801F78003BD107006F00B10010
:10CF900020002000801F780080EA2000801F780099
:10CFA0000009200000004700801F780032D10700F0
:10CFB0006F00B10020002000801F780080E020007A
:10CFC000801F78000009200000004700801F7800C3
:10CFD00029D107006F00B10010002000801F7800E9
:10CFE00060E02000801F780000092000000047005A
:10CFF000801F780020D107006F00B10020002000C2
:10D00000801F7800A0EC2000801F7800000920001D
:10D0100000004700801F780017D107006F00B100A3
:10D0200020002000801F780000E42000801F78008E
:10D030000009200000004700801F78000ED1070083
:10D040006F00B10020002000801F7800C0ED20009C
:10D05000801F78000009200000004700801F780032
:10D0600005D107006F00B10020002000801F78006C
:10D07000C0E32000801F7800000920000000470066
:10D08000801F7800FCD007006F00B1002000200056
:10D09000801F780000EE2000801F7800000920002B
:10D0A00000004700801F7800F3D007006F00B10038
:10D0B00020002000801F780040EE2000801F7800B4
:10D0C0000009200000004700801F7800EAD0070018
:10D0D0006F00B10020002000801F780080E4200055
:10D0E000801F78000009200000004700801F7800A2
:10D0F000E1D007006F00B10020002000801F780001
:10D1000040E42000801F7800000920000000470054
:10D11000801F7800D8D007006F00B10020002000E9
:10D12000801F780040E32000801F78000009200065
:10D1300000004700801F7800CFD007006F00B100CB
:10D1400020002000801F780080EE2000801F7800E3
:10D150000009200000004700801F7800C6D00700AB
:10D160006F00B10020002000801F780080E32000C5
:10D17000801F78000009200000004700801F780011
:10D18000BDD007006F00B10020002000801F780094
:10D1900060EC2000801F780000092000000047009C
:10D1A000801F7800B4D007006F00B100100020008D
:10D1B000801F7800A0E52000801F78000009200073
:10D1C00000004700801F7800ABD007006F00B1005F
:10D1D00010002000801F7800E0E52000801F78000C
:10D1E0000009200000004700801F7800A2D007003F
:10D1F0006F00B10010002000801F780020EA20009E
:10D20000801F78000009200000004700801F780080
:10D2100099D007006F00B10010002000801F780037
:10D2200000D22000801F7800000920000000470085
:10D23000801F780090D007006F00B1001000200020
:10D24000801F780020DD2000801F7800000920006A
:10D2500000004700801F780087D007006F00B100F2
:10D2600010002000801F7800C0EE2000801F780092
:10D270000009200000004700801F78007ED00700D2
:10D280006F00B10020002000801F7800E0EE200039
:10D29000801F78000009200000004700801F7800F0
:10D2A00075D007006F00B10020002000801F7800BB
:10D2B00020EF2000801F78000009200000004700B8
:10D2C000801F78006CD007006F00B10010002000B4
:10D2D000801F7800E0E92000801F7800000920000E
:10D2E00000004700801F780063D007006F00B10086
:10D2F000F074800000758800347080006000520077
:10D300000C0035007609200064E0200014001300B2
:10D3100008003C00A6D72000CFB3DE00E4D02000F8
:10D320003400130024801B0002003500466A04000C
:10D33000000000000000200001242400407288004A
:10D34000517288000000200001222400E071880052
:10D35000F171880000002000011724000077880088
:10D36000117788000000200001122400007288005C
:10D37000117288000000200001102400207788002E
:10D38000317788000000200001F82300E076880053
:10D39000F176880000002000010A24002072880035
:10D3A000317288000000200041232400407788006B
:10D3B000517788000000200001122400C07188000D
:10D3C000D1718800B0042000307088000000240073
:10D3D000C159240050768800617688006066260076
:10D3E00061FA23004070880051708800100020000E
:10D3F000D072880010002000F07288000000200029
:10D40000812C2400A0718800B171880000002800E0
:10D41000414D2400307688004176880090C2250076
:10D42000F1D8230040758800517588000000200065
:10D430006149240070768800817688001000200001
:10D44000107588002004200000698800100020006A
:10D45000906E8800F000200060778800503A2F001E
:10D4600061982300707788008177880080392100D7
:10D4700041D9230090778800A17788000000200020
:10D480000075880000002000F07488000000200073
:10D49000010E240090758800A1758800000020000E
:10D4A000010E2400D0758800E1758800407080006E
:10D4B00051708000A06E8800B16E880030708000CE
:10D4C000C06E88003470800080DD2000610842005A
:10D4D00000002000503F9800A007200000004700F7
:10D4E000100278006C00520016003D00A6072000D4
:10D4F00006034700160078004202DD0040D62000F7
:10D500000402400000002000000A780006007800B5
:10D51000100078004202DD0040D6200004004000E8
:10D520006202400000002000000A78001400200081
:10D53000A007200000004700100842006C6A0400A9
:10D540000000000000002000100E8800701A260065
:10D55000200E880080002800000E880060EA20006D
:10D56000D00E8800D00E8000C00E8800C00E800053
:10D57000B00E8800E06A2000801F7800700B200049
:10D58000801F78003CFA07004F00B10085E40700D7
:10D59000D20DF800F0922F00801F780020E62000C6
:10D5A000801F7800E9F307006F00B10020E620003B
:10D5B000801F78000AF407002F00B10065004700C3
:10D5C000801F780006F407002F00B100E04620001D
:10D5D000801F7800A0072000801F780026FA07002F
:10D5E0004F00B1002CF4070074004700801F780042
:10D5F000FBF307002F00B100E01E2100801F780020
:10D60000801E2000801F78001BFA07004F00B10029
:10D6100020002000503F9800A00720000000470095
:10D62000100278006000520018003400A0072000AB
:10D63000000047001000780061005000503F980043
:10D64000801F780080932F00801F780040D9200031
:10D65000801F7800BDF307006F00B10040D92000A3
:10D66000801F7800B4D207002F00B100E0CE220066
:10D67000801F7800404C2000801F7800FEF90700D2
:10D680004F00B1000C6B04000000000045E40700EF
:10D6900004402000E0202000100872000400280050
:10D6A000C020200010087200F0012000801F7800C8
:10D6B00059CD07002F00B100A0002000801F780086
:10D6C00055CD07002F00B100E00420000000470006
:10D6D000801F780098D207002F00B10068CD0700A6
:10D6E00060025000020035006E6B04000000000074
:10D6F0007BCD07000004E00003003A000060FE005C
:10D70000786B040000000000E08E2000801F78008D
:10D71000400F2000801F7800D7F907004F00B100AC
:10D7200020E40700E0682000801F780060002000EF
:10D73000801F7800D0F907004F00B100D6F3070032
:10D740007006200000004700801F7800B2E6070046
:10D750002F00B100E0462000801F7800A0072000C5
:10D76000801F7800C4F907004F00B10010002000AE
:10D77000801F7800F1E607002F00B100E04620008E
:10D78000801F7800A0072000801F7800BAF90700EA
:10D790004F00B100B006200000004700801F780055
:10D7A0009DE607002F00B100100720000000470091
:10D7B000801F780098E607002F00B100D068800035
:10D7C000CF80DE000081EB00F4F90700E262250063
:10D7D00043CD23004CFA07003097980041979800FA
:10D7E0007075880081758800E0688000CF80DE0059
:10D7F0000081EB00E9F90700E262250043CD230038
:10D8000041FA0700B0758800C17588003E9090000D
:10D81000CE90900000027800810278000000200085
:10D82000811024000401780085017800C3FA070004
:10D830000000E00002003C00000020000100370072
:10D84000100020000000E000060032000000200070
:10D85000010E240090758800A17588003A6C0400C0
:10D8600000000000000020000112240090758800D4
:10D87000A1758800B4758000C57580000000200087
:10D88000811024000401780085017800ABFA0700BC
:10D890000000E00002003C00000020000100370012
:10D8A000100020000000E000060032000000200010
:10D8B000010E2400D0758800E1758800926C040088
:10D8C00000000000B4758000C5758000D0CC2C002D
:10D8D000C1142400040178008501780097FA07003C
:10D8E0000000E00002003C000000200001003700C2
:10D8F000100020000000E0000600320000002000C0
:10D9000001122400D0758800E1758800926C040033
:10D91000000000000000200001152400D0758800E0
:10D92000E175880000002000503F980000002000B2
:10D9300000879800EACC07000004E000570132009D
:10D940000060FE00CECC0700603F980060025000EF
:10D950005001350036062000A407200004024700CD
:10D96000140013000600340000002000503F98000F
:10D9700000002000008798004A6F040000000000AB
:10D98000286F04000000000000002000503F9800B5
:10D9900010002000008798004A6F0400000000007B
:10D9A00080F02000A6072000060347001602400072
:10D9B00000002000004A780010002000160B4000F4
:10D9C0004A6F04000000000084F02000A00720003F
:10D9D000000047001002420000002000004A7800CA
:10D9E000000820000000470010027800600052008C
:10D9F00004013200000020000087980080F0200021
:10DA0000801F7800CACE07002F00B10060025000CE
:10DA1000FC003400A0708000B17080002075880088
:10DA200031758800F46A8000056B8000126F8000F9
:10DA3000236F8000040078008500780044FA070016
:10DA4000A0708800B1708800247580003575800052
:10DA500004017800850178003DFA070020758800F0
:10DA6000317588002008200000004700100378006E
:10DA7000C4D32000140053005800320014002000CA
:10DA80004008200000004700100842001400200059
:10DA9000600820000000470010084200A6708000C7
:10DAA000B770800084082000040247003401780029
:10DAB000A4017800060078008700780024FA0700A7
:10DAC0007072880081728800866A8000976A800080
:10DAD000C40820000402470034017800A401780043
:10DAE000060078008700780019FA0700A072880005
:10DAF000B1728800000278008102780000002000E6
:10DB00004133240004017800850178004EFA0700B3
:10DB10000000E00002003500000020000100370096
:10DB2000100020000000E0000B003200A472800012
:10DB3000B572800002002000433B240004007800FE
:10DB40008500780002FA0700A0728800B172880090
:10DB5000DA6D040000000000A4728000B57280003D
:10DB60000000200041332C0004017800850178007A
:10DB7000F2F907000000E00002003C000000200075
:10DB800001003700100020000000E0000900320012
:10DB9000A4728000B572800000002000413B240088
:10DBA00004017800850178002CFA0700A072880033
:10DBB000B1728800E069800010879800A070800032
:10DBC000B17080004087980051879800806A80007B
:10DBD000916A8000608798007187980024708000A7
:10DBE0006000520003003A006AD10700026F04008F
:10DBF0000000000000002000801F7800F8D6070019
:10DC00002F00B10064688000600052000C003A00F0
:10DC1000546880006000520009003A00400820006B
:10DC200000004700901F780010002000801F78003F
:10DC300092D807004F00B1002E6E040000000000D3
:10DC40004008200000004700901F780000002000DE
:10DC5000801F780089D807004F00B1000000200025
:10DC600020879800647780006000520065003400CF
:10DC7000600820000000470010037800C4EE200078
:10DC8000140053005F00350000002000308798002A
:10DC9000646A8000756A80000000200001F02300A3
:10DCA0000401780085017800E7F907000000E00032
:10DCB00002003400000020000100370010002000A6
:10DCC0000000E00007003A00E007200000004700E5
:10DCD000100278006000520002003200026F04005F
:10DCE00000000000400920000000470030037800D9
:10DCF000A003780044FF2F00F50720000400530024
:10DD000005805B003F003E0000242400F10020005D
:10DD1000F2698000CF91DE0086FA070046D5200028
:10DD200036024000A6824800349798004597980034
:10DD300000102E00515F2000026A8000CF91DE00AB
:10DD40007CFA07003E929000CE92900000024200C2
:10DD500081824A008009200000004700101842001C
:10DD600010904A00E00720000000470010027800F1
:10DD70006000520018003A0020002000CF80DE0032
:10DD80004409200004024700141A100014921800DD
:10DD900010002000801F7800E007200000004700EE
:10DDA000801F7800841F7800D0E507006F00B10065
:10DDB00020002000801F780080092000000047001C
:10DDC000801F78004009200000004700801F780075
:10DDD000C6E507006F00B100E00720000000470023
:10DDE0001000780061004000703F9800801F7800AC
:10DDF0004009200000004700801F7800CED90700AE
:10DE00004F00B1004A6F040000000000000820002D
:10DE10000000470010027800600052000A00320043
:10DE200080F02000A60720000603470016024000ED
:10DE3000C00720000000470010407800004A78002A
:10DE400010002000160B40004A6F04000000000084
:10DE500046022000C40720000402470014001300FB
:10DE6000C9FE3200C0072000000047001002780001
:10DE70006D005200CAFE3200C007200000004700BB
:10DE8000100278006A005200CFFE3200066F0400D4
:10DE9000000000009A6C04000000000060D2200026
:10DEA0001042780064405200CD00360064D2200059
:10DEB00000002000004A7800D0688000CF80DE009B
:10DEC0000081EB0035F80700E262250043CD230016
:10DED0008DF8070074758000857580000401780056
:10DEE000850178005DF9070002002000030024008E
:10DEF00019FA07007075880081758800E068800055
:10DF0000CF80DE000081EB0024F80700E2622500EC
:10DF100043CD23007CF80700B4758000C5758000F0
:10DF200004017800850178004CF907000200200008
:10DF30000300240008FA0700B0758800C175880046
:10DF4000000A200000004700100278006200520022
:10DF5000020035000000200000979800C40920004E
:10DF600004024700060A2000060347001600780056
:10DF70004100DD0000024200F0688000000A7800E5
:10DF800010002000160B4000000020002097980091
:10DF90000000200010979800200A20000000470091
:10DFA000100278006200520011003D00C4092000F8
:10DFB00004024700200A20000000470010007800FB
:10DFC0004100DD000000420010027800400A2000FD
:10DFD000000047001008420014002000200A200022
:10DFE0000000470010084200CC6F04000000000051
:10DFF0002E909000CF80DE000081EB00E7F7070055
:10E000000200200003002400D3F90700927780006B
:10E01000A37780003CF80700F0758800017688003F
:10E02000000278008102780090768000A17680005E
:10E03000040178008501780003F907000000E00082
:10E040000200350000002000010037001000200011
:10E050000000E00004003200F075800001768000CE
:10E0600090768800A1768800106980002169800080
:10E070000001EB00C9F7070072778000837780000A
:10E0800021F80700107688002176880006AF20006E
:10E09000CFB3DE0024D120003400130024801B0005
:10E0A00014003D00207080000000E00011003200EC
:10E0B000546880006100520007003A000000200010
:10E0C0005068880010002000106B8800B5E1070040
:10E0D00076700400000000000000200060688800E6
:10E0E00010002000806E880093D90700EE700400B5
:10E0F000000000001000200060688800C63E21007B
:10E10000CFB3DE0024D120003400130024801B0094
:10E110000400340060EA2000CF80DE0090688800B0
:10E12000A1688800C6252100CFB3DE0024D12000DD
:10E130003400130024801B0008003400846E80002B
:10E140006100520003003A0096E107000000200041
:10E15000806E8800EE700400000000004619210067
:10E16000CFB3DE0024D120003400130024801B0034
:10E170000F003400846E80006100520003003A00FA
:10E1800088E1070000002000806E8800546880004D
:10E190006000520003003A00100020005068880020
:10E1A000DDE3070041F10700EE700400000000000D
:10E1B000546880006100520005003A000000200011
:10E1C0005068880077E10700EE700400000000004E
:10E1D00010002000806E880057D907000BF7070059
:10E1E0009A6C0400000000000080FA00FFFF370076
:10E1F0003235FF00312CFF003131FF003532FF0096
:10E200003030FF000000FF000000FF000000FF00B2
:10E210000000FF000000FF000000FF000000FF0002
:10E220000000FF000000FF000000FF00003CFF00B6
:10E230000A25FF003031FF00306CFF00750AFF0037
:10E240000025FF00382EFF003666FF002C25FF005A
:10E25000382EFF003666FF002C25FF00640AFF0001
:10E260000047FF005052FF004D43FF000047FF00F2
:10E270005047FF004741FF000047FF005047FF00A5
:10E280005356FF000050FF00494EFF004700FF00BB
:10E29000504FFF004E47FF000A00FF004745FF00B8
:10E2A000544CFF004F47FF00003EFF000A00FF00F4
:10E2B0005365FF007474FF00696EFF006720FF0064
:10E2C000484FFF004D45FF002025FF002D33FF0084
:10E2D0006400FF00484FFF004D45FF00206EFF0027
:10E2E0006F74FF002073FF006574FF0000FFFF00E4
:10E2F0000000FF000000FF00C4FFFF007F3FFF00A1
:10E3000080EFFF00FFBEFF0090E1FF00A93EFF008D
:10E31000EC82FF0076BEFF0082ADFF002B3EFF00C7
:10E320000E3CFF00C3BDFF0087D1FF00133DFF007F
:10E330004178FF00D3BBFF000000FF00803FFF00DB
:10E340001872FF00313FFF00F0FDFF00753EFF0037
:10E350004758FF00633DFF005895FF001D3CFF003C
:10E3600082C4FF00AE3AFF00A878FF002139FF0009
:10E37000EF93FF008037FF00A092FF00A735FF005A
:10E380004656FF001534FF00ECF3FF004A48FF003B
:10E390003595FF0095C7FF0017C1FF00DC45FF0062
:10E3A000FDDBFF006DC3FF0072B3FF003340FF00D1
:10E3B0002B34FF000148FF007F9DFF00B045FF00A8
:10E3C000E7FFFF00D942FF000000FF00803FFF0091
:10E3D000063CFF000442FF007D9FFF006A42FF00F1
:10E3E0005C90FF000142FF00604DFF00BB40FF005A
:10E3F00051ECFF00473EFF00DE8DFF001FBBFF001A
:10E40000063CFF000442FF00C059FF008B42FF00A2
:10E410007404FF004442FF00F99BFF004F41FF00DE
:10E420000000FF00803FFF001B5BFF003958FF002A
:10E43000001BFF005B37FF00396DFF004155FF00F7
:10E44000544FFF005049FF004C4FFF005400FF00A5
:10E450001B5BFF00307AFF001B5BFF002564FF00A1
:10E460003B25FF006478FF00001BFF005B34FF00CA
:10E470007A1BFF005B25FF00643BFF002564FF0063
:10E480007800FF001B5BFF00307AFF001B5BFF0082
:10E490002564FF003B25FF006448FF000025FF00C6
:10E4A0003032FF00643AFF002530FF003264FF0085
:10E4B0001B5BFF00347AFF002530FF003264FF0051
:10E4C0002055FF005443FF000025FF003032FF00BD
:10E4D000643AFF002530FF003264FF001B5BFF0041
:10E4E000347AFF002530FF003264FF000025FF0072
:10E4F0002336FF002E31FF00661BFF005B31FF005B
:10E500007A6BFF007068FF000025FF002336FF00D4
:10E510002E31FF00661BFF005B31FF007A6DFF00AC
:10E520007068FF000025FF002336FF002E31FF003A
:10E53000661BFF005B31FF007A6DFF000025FF00C6
:10E540002336FF002E31FF00661BFF005B31FF000A
:10E550007A66FF007400FF001B5BFF00307AFF004B
:10E560002563FF002563FF000025FF002335FF0022
:10E570002E32FF00661BFF005B31FF007A56FF0062
:10E580000025FF002335FF002E32FF00661BFF0031
:10E590005B31FF007A56FF001B5BFF003639FF003E
:10E5A0006D1BFF005B34FF007A20FF004558FF0021
:10E5B0005400FF002523FF00352EFF003166FF00C9
:10E5C0001B5BFF00317AFF004100FF002535FF0093
:10E5D0002E30FF00661BFF005B31FF007A6DFF00ED
:10E5E0004168FF000025FF00342EFF003066FF0069
:10E5F0001B5BFF00317AFF006D00FF002523FF0049
:10E60000342EFF003266FF001B5BFF00317AFF00F3
:10E610006D6CFF000025FF00352EFF003066FF0007
:10E620001B5BFF00317AFF006D00FF002523FF0018
:10E63000352EFF003266FF001B5BFF00317AFF00C2
:10E640006D6CFF00001BFF005B34FF007A53FF007E
:10E650005045FF004544FF00201BFF005B30FF00DA
:10E660007A25FF002336FF002E31FF00661BFF00D6
:10E670005B31FF007A6BFF007068FF00001BFF003A
:10E680005B34FF007A20FF002041FF004C54FF0064
:10E69000201BFF005B30FF007A25FF002336FF00C0
:10E6A0002E31FF00661BFF005B31FF007A6DFF001B
:10E6B000001BFF005B34FF007A52FF00414EFF0059
:10E6C0004745FF00201BFF005B30FF007A25FF005D
:10E6D000362EFF003066FF001B5BFF00317AFF0023
:10E6E0006D00FF001B5BFF00347AFF005350FF00FA
:10E6F0004545FF004420FF001B5BFF00307AFF0010
:10E700002523FF00362EFF003166FF001B5BFF0054
:10E71000317AFF006D70FF006800FF001B5BFF0097
:10E72000347AFF002020FF00414CFF005420FF00FE
:10E730001B5BFF00307AFF002523FF00362EFF0011
:10E740003166FF001B5BFF00317AFF006674FF003B
:10E75000001BFF005B34FF007A52FF00414EFF00B8
:10E760004745FF00201BFF005B30FF007A25FF00BC
:10E770002336FF002E32FF00661BFF005B31FF00D7
:10E780007A6DFF006C00FF001B5BFF00347AFF0016
:10E790002043FF005552FF005220FF001B5BFF008B
:10E7A000307AFF002523FF00362EFF003166FF0080
:10E7B0001B5BFF00317AFF004100FF001B5BFF0085
:10E7C0003635FF006D25FF003264FF001B5BFF0044
:10E7D0003639FF006D1BFF005B34FF007A20FF001D
:10E7E0005341FF005453FF000025FF003264FF0037
:10E7F0001B5BFF00347AFF002053FF004154FF00F1
:10E800005300FF002523FF003130FF002E36FF00AC
:10E81000661BFF005B34FF007A25FF006300FF00EA
:10E820002523FF003130FF002E36FF00661BFF005E
:10E830005B34FF007A25FF006300FF001B5BFF00D5
:10E84000347AFF004844FF004F50FF00201BFF00B8
:10E850005B30FF007A25FF00232DFF00362EFF00DE
:10E860003166FF000025FF003033FF006400FF0029
:10E870002025FF007320FF00001BFF005B37FF0017
:10E88000346DFF002530FF00332EFF003066FF009F
:10E890000025FF003033FF002E30FF006600FF0030
:10E8A000201BFF005B37FF00316DFF002573FF0069
:10E8B0001B5BFF003639FF006D20FF000020FF00CA
:10E8C0002573FF002000FF002025FF007320FF00BC
:10E8D00000C4FF002563FF001B5BFF00347AFF00CC
:10E8E000201BFF005B30FF007A00FF00C425FF0003
:10E8F000631BFF005B34FF007A20FF001B5BFF00FF
:10E90000307AFF000025FF003032FF006420FF0056
:10E91000001BFF005B38FF005800FF001B5BFF007F
:10E920003658FF00001BFF005B37FF005800FF0058
:10E930001B5BFF003758FF00001BFF005B34FF002C
:10E940007A4CFF004F53FF00201BFF005B30FF009D
:10E950007A00FF005045FF00414BFF002056FF00AA
:10E96000414CFF005545FF005300FF001B5BFF00BB
:10E970003131FF005800FF001B5BFF003132FF0008
:10E980005800FF001B5BFF003132FF005800FF0002
:10E990001B5BFF003132FF005800FF001B5BFF00D4
:10E9A0003132FF005800FF001B5BFF003958FF00A9
:10E9B000001BFF005B35FF005800FF001B5BFF00E2
:10E9C0003131FF005800FF001B5BFF003131FF00B9
:10E9D0005800FF001B5BFF003958FF0000C0FF001C
:10E9E000A000FF00C0A0FF0000C3FF00BF00FF00A9
:10E9F000C480FF0000C0FF00A000FF00C480FF0033
:10EA000000C3FF00BF00FF00C0A0FF00001BFF000D
:10EA10005B34FF007A00FF002D2DFF002000FF0077
:10EA20001B5BFF00324AFF00001BFF005B31FF0051
:10EA30007A1BFF005B25FF00643BFF002564FF009D
:10EA40007800FF00204DFF004158FF005241FF00B9
:10EA50004E47FF004520FF002020FF00201BFF0045
:10EA60005B30FF007A25FF00362EFF003066FF0086
:10EA70002000FF00204CFF004F57FF00414CFF00DB
:10EA80005452FF004154FF00494FFF00201BFF007C
:10EA90005B30FF007A25FF00362EFF003266FF0054
:10EAA0002000FF002056FF00414CFF004944FF00BA
:10EAB0004844FF004F50FF002020FF00201BFF00B4
:10EAC0005B30FF007A25FF00362EFF003166FF0025
:10EAD0002000FF00204DFF00494EFF005641FF007F
:10EAE0004C49FF004420FF002020FF00201BFF00B6
:10EAF0005B30FF007A25FF003664FF002000FF0036
:10EB00002053FF00484FFF005748FF004F4DFF00C4
:10EB1000454CFF00494DFF00201BFF005B30FF000C
:10EB20007A25FF00362EFF003066FF002000FF0030
:10EB30002052FF004F43FF004C49FF004D49FF00AA
:10EB40005420FF002020FF00201BFF005B30FF004F
:10EB50007A25FF00362EFF003166FF002000FF00FF
:10EB60002052FF004F43FF005354FF004550FF0069
:10EB70004741FF00494EFF00201BFF005B30FF00B4
:10EB80007A25FF00362EFF003066FF002000FF00D0
:10EB90002041FF005052FF004F43FF004741FF005C
:10EBA000494EFF002020FF00201BFF005B30FF00CC
:10EBB0007A25FF00362EFF003166FF002000FF009F
:10EBC0002052FF004F54FF004C49FF004D49FF0009
:10EBD0005420FF002020FF00201BFF005B30FF00BF
:10EBE0007A25FF00362EFF003166FF002000FF006F
:10EBF0002052FF004F54FF005354FF004550FF00C8
:10EC00004741FF00494EFF00201BFF005B30FF0023
:10EC10007A25FF00362EFF003066FF002000FF003F
:10EC20002041FF005052FF004F54FF004741FF00BA
:10EC3000494EFF002020FF00201BFF005B30FF003B
:10EC40007A25FF00362EFF003166FF002000FF000E
:10EC50002053FF005045FF004544FF004C4FFF008C
:10EC6000574CFF00494DFF00201BFF005B30FF00A9
:10EC70007A25FF00362EFF003166FF002000FF00DE
:10EC80002043FF005255FF004953FF004541FF005C
:10EC90004C54FF002020FF00201BFF005B30FF00D2
:10ECA0007A25FF00362EFF003066FF002000FF00AF
:10ECB000204DFF004158FF00414CFF005443FF002E
:10ECC0004847FF002020FF00201BFF005B30FF00B3
:10ECD0007A25FF00362EFF003066FF002000FF007F
:10ECE000204DFF004158FF004844FF004743FF000C
:10ECF0004847FF002020FF00201BFF005B30FF0083
:10ED00007A25FF00362EFF003066FF002000FF004E
:10ED1000204DFF004148FF005741FF00524EFF00C9
:10ED2000494EFF004720FF00201BFF005B30FF0023
:10ED30007A25FF00362EFF003066FF002000FF001E
:10ED40002045FF004C45FF005345FF005256FF0091
:10ED50004F44FF004952FF00201BFF005B30FF00C3
:10ED60007A25FF003673FF002000FF002052FF00CD
:10ED70004452FF005345FF005256FF004F44FF002E
:10ED80004952FF00201BFF005B30FF007A25FF0087
:10ED90003673FF002000FF002055FF004E49FF00A2
:10EDA0005453FF002020FF002020FF002020FF0000
:10EDB0002020FF002538FF007320FF000020FF0007
:10EDC000414DFF005053FF005A45FF00524FFF00D6
:10EDD0002020FF002020FF001B5BFF00307AFF0097
:10EDE0002536FF006420FF000020FF005649FF0089
:10EDF0004445FF004F4DFF004F44FF004520FF00FA
:10EE00002020FF002025FF003873FF002000FF00B6
:10EE1000204CFF004F47FF005045FF005249FF00C4
:10EE20004F44FF002020FF00201BFF005B30FF004D
:10EE30007A25FF003664FF002000FF002048FF0015
:10EE40004F4DFF00454CFF004F43FF002020FF00C7
:10EE50002020FF002020FF002538FF007320FF0046
:10EE60000020FF004D41FF00484DFF00554CFF00C2
:10EE70005420FF002020FF00201BFF005B30FF001C
:10EE80007A25FF00372EFF003566FF002000FF00C7
:10EE90002041FF004D50FF004D55FF004C54FF0036
:10EEA0002020FF002020FF00201BFF005B30FF0020
:10EEB0007A25FF00362EFF003366FF002000FF009A
:10EEC0002053FF004146FF00455AFF004F4EFF0010
:10EED0004520FF002020FF00201BFF005B30FF00CB
:10EEE0007A25FF003664FF002000FF002056FF0057
:10EEF0004F4CFF005431FF004C4FFF005741FF00C3
:10EF0000524EFF00201BFF005B30FF007A25FF0000
:10EF10003673FF002000FF002053FF004156FF0022
:10EF20004520FF00434FFF004E46FF004947FF00CA
:10EF3000201BFF005B30FF007A25FF003673FF00C7
:10EF40002000FF004E4FFF005200FF005245FF001F
:10EF50005600FF004E4FFF005200FF005245FF00D9
:10EF60005600FF004D45FF005452FF004943FF008B
:10EF70000049FF004D50FF004552FF004941FF008E
:10EF80004C00FF005041FF004C00FF004E54FF00BA
:10EF90005343FF000053FF004554FF000055FF009E
:10EFA0004E53FF004554FF00004FFF004646FF0050
:10EFB0000020FF004F4EFF00002AFF000044FF002A
:10EFC0004F4EFF004500FF002530FF003278FF0064
:10EFD0000024FF00504DFF00544BFF002573FF003D
:10EFE0002A25FF00730DFF000A00FF003331FF00E8
:10EFF000342CFF00302CFF00312CFF00302CFF00A0
:10F00000312CFF00302CFF000031FF000030FF00EA
:10F01000002CFF00302CFF00302CFF00302CFF00B4
:10F02000302CFF00302CFF00302CFF00302CFF0074
:10F03000302CFF00302CFF00302CFF003000FF0090
:10F040000000FF00803FFF00CDCCFF00CC3DFF0063
:10F050000AD7FF00233CFF006F12FF00833AFF0036
:10F0600017B7FF00D138FF00ACC5FF002737FF00FE
:10F07000BD37FF008635FF0095BFFF00D633FF0088
:10F0800077CCFF002B32FF005F70FF008930FF005C
:10F09000FFE6FF00DB2EFF0008E5FF003C1EFF003F
:10F0A0006042FF00A20DFF000000FF00803FFF0054
:10F0B0000000FF002041FF000000FF00C842FF00E9
:10F0C0000000FF007A44FF000040FF001C46FF00E4
:10F0D0000050FF00C347FF000024FF007449FF00F9
:10F0E0008096FF00184BFF0020BCFF00BE4CFF00C5
:10F0F000286BFF006E4EFF00F902FF001550FF0065
:10F10000EC78FF00AD60FF00CAF2FF004971FF001C
:10F110000100FF000000FF000A00FF000000FF00E8
:10F120006400FF000000FF00E803FF000000FF0094
:10F130001027FF000000FF00A086FF000100FF0075
:10F140004042FF000F00FF008096FF009800FF0084
:10F1500000E1FF00F505FF0000CAFF009A3BFF0039
:10F160000100FF000000FF001000FF000000FF0092
:10F170000001FF000000FF000010FF000000FF0082
:10F180000000FF000100FF000000FF001000FF0072
:10F190000000FF000001FF000000FF000010FF0062
:10F1A0000100FF000000FF000800FF000000FF005A
:10F1B0004000FF000000FF000002FF000000FF0011
:10F1C0000010FF000000FF000080FF000000FF00B3
:10F1D0000000FF000400FF000000FF002000FF000F
:10F1E0000000FF000001FF000000FF000008FF001A
:10F1F0000000FF000040FF000000FF000000FF00D3
:10F200003031FF003233FF003435FF003637FF0066
:10F210003839FF004142FF004344FF004546FF00EC
:10F220000030FF003132FF003334FF003536FF007D
:10F230003738FF003961FF006263FF006465FF003B
:10F240006600FF00286EFF00756CFF006C29FF0050
:10F25000001BFF005B25FF00646DFF00001BFF002B
:10F260005B31FF00363BFF002564FF007600FF00A6
:10F270004750FF00532FFF004F53FF004420FF0073
:10F280005354FF004152FF005455FF005020FF002F
:10F290002564FF000048FF004F4DFF004500FF00C0
:10F2A0001B5BFF003231FF003B30FF00761BFF008D
:10F2B0005B33FF00323BFF003176FF00001BFF0095
:10F2C0005B31FF007A44FF007261FF00676FFF004F
:10F2D0006E4FFF005344FF002056FF006572FF0091
:10F2E0007369FF006F6EFF002034FF002E36FF00B1
:10F2F0002032FF00382FFF003131FF002F32FF0096
:10F300003030FF003720FF00436FFF007079FF00AF
:10F310007269FF006768FF007420FF004461FF000E
:10F320006E69FF00656CFF002057FF006565FF00F8
:10F330000057FF006169FF007469FF006E67FF00FE
:10F340002066FF006F72FF002047FF005053FF0050
:10F350002064FF006174FF006120FF002E2EFF007B
:10F360002E00FF003030FF003000FF003331FF007F
:10F37000332CFF003100FF003232FF00302CFF0041
:10F380003230FF003000FF00FFFFFF00FFFFFF00F3
:0200000401F009
:10000000F6FF0000F4FF00007F7A0000FFFFFF0012
:0C001000FFFFFF00FFFF0000FFFF0000EB
:00000001FF
